:100000000C941E060C946F280C949C280C944606A5
:100010000C9446060C9446060C9446060C94460630
:100020000C9446060C9446060C9432130C94460627
:100030000C9446060C9446060C9446060C94460610
:100040000C94C9280C9446060C94B72C0C94FA2CEA
:100050000C9446060C9446060C9446060C944606F0
:100060000C9446060C944606E218441923192619E6
:1000700029192C192F193219351944193E19761AD4
:10008000781A781A761A781A781A781A781A781AE2
:10009000781A781A781A781A781A781A781A781AD0
:1000A000FC19781A781A781A781A781A6D19781A49
:1000B000781A781A781A781A781A781A781A781AB0
:1000C000781A781A781A781A781A781A081A081A80
:1000D000081A081A081A081A081A081A081A781AA0
:1000E000781A781A781A781A781A6D19071A071A6E
:1000F000071A071A781A151A1B1A211A271A2D1A05
:10010000331A391A3F1A491A531A5D1A671AAE1967
:100110007019781A781A781A781AFC19781A781AD5
:10012000781A781A781A781A781A781A061A061A23
:10013000061A061A781A151A1B1A211A271A2D1AC6
:10014000331A391A3F1A491A531A5D1A671AAE1927
:100150007019781A781A781A781AFC19AB1AAB1A2F
:10016000AB1AAB1AAB1AAB1AAB1AAB1AAB1AAB1A67
:10017000AB1AAB1AAB1AC21BC21BC21BC21BC21BDF
:10018000C21BF01AFA1A041B0E1B6C1B761B851B74
:10019000961B1E1D331D3F1D481D571D7C1D851DB3
:1001A000CE1D971DE220E820EE20F5200321252119
:1001B0004321456E746572206D656E752E2E2E007E
:1001C000546F67676C6564206D6963726F50504D42
:1001D00000546F67676C656420696E76657274653C
:1001E000642050504D2100546F67676C6564205443
:1001F00058206D7574696E672100546F67676C6570
:10020000642074656C656D65747279210050726F3D
:10021000746F636F6C206572726F72207769746897
:100220002052580054696D656F7574207768656E4B
:1002300020636F6E6E656374696E6720746F205201
:100240005800507265737320616E79206B65792058
:10025000746F2063616E63656C00436F6E6E6563DF
:1002600074696E6720746F2052582C20706F776508
:100270007220757020746865205258202877697440
:10028000682062696E6420706C7567206966206EF4
:100290006F74207573696E6720616C776179732064
:1002A00062696E642900546F67676C656420276912
:1002B0006D6D656469617465206F75747075742700
:1002C00000546F67676C65642027736C61766520E6
:1002D0006D6F64652700546F67676C6564202761E4
:1002E0006C776179732062696E642700546F676769
:1002F0006C65642050504D206368616E6E656C20A3
:100300006C696D69740053657420525353492069B8
:100310006E6A656374696F6E206368616E6E656C8A
:100320002028303D3D64697361626C652900536526
:10033000742050504D206D696E696D756D20737914
:100340006E630053657420626561636F6E20696E31
:1003500074657276616C0053657420626561636FC9
:100360006E2064656C617900536574206265616319
:100370006F6E206672657175656E637920696E2097
:10038000487A3A20303D64697361626C652C205074
:10039000783D504D52206368616E6E656C20782CFC
:1003A0002046783D465253206368616E6E656C202E
:1003B00078005365742050574D2073746F7020641B
:1003C000656C61792028302064697361626C6564B2
:1003D0002C20312D323535203D3D20302E317320FB
:1003E0002D2035306D696E29005365742050504DB5
:1003F0002073746F702064656C61792028302064EC
:10040000697361626C65642C20312D323535203D75
:100410003D20302E3173202D2035306D696E29003E
:10042000536574206661696C736166652064656CF0
:1004300061792028302064697361626C65642C20C6
:10044000312D323535203D3D20302E3173202D2089
:1004500035306D696E29002A2A2A2A2A2A2A2A2A50
:100460002A2A2A2A2A2A2A2A2A2A2A2A2A2A2A2AEC
:100470002A2A2A2A0052582041636B6564202D20C5
:1004800072657665727420737563636573736675E0
:100490006C21002A2A2A2A2A2A2A2A2A2A2A2A2AAD
:1004A0002A2A2A2A2A2A2A2A2A2A2A2A2A2A2A2AAC
:1004B000002A2A2A2A2A2A2A2A2A2A2A2A2A2A2AC6
:1004C0002A2A2A2A2A2A2A2A2A2A2A2A2A2A00528E
:1004D000582041636B6564202D20757064617465DC
:1004E000207375636365737366756C21002A2A2A0D
:1004F0002A2A2A2A2A2A2A2A2A2A2A2A2A2A2A2A5C
:100500002A2A2A2A2A2A2A2A2A2A0056616C696457
:100510002063686F69636573206172653A205B319F
:100520005D2D5B31365D20286368616E6E656C20E1
:10053000312D31362900536574206F7574707574D0
:1005400020666F7220706F727420005B585D2061AE
:10055000626F7274206368616E67657320616E6498
:10056000206578697420525820636F6E6669670051
:100570005B535D20736176652073657474696E6783
:100580007320746F205258005B525D20726576654F
:1005900072742052582073657474696E6773207486
:1005A0006F2064656661756C747300557365206EA9
:1005B000756D62657273205B312D445D20746F2010
:1005C0006564697420706F727473205B452D515D92
:1005D00020666F722073657474696E677300202DD6
:1005E00020726563656976657220636F6E66696700
:1005F000757261746F722C20727820737720000AF4
:100600000A6F70656E4C52536E67200053657420FC
:1006100073657269616C2062617564726174653AB8
:10062000200056616C69642063686F696365733A82
:100630002031202D20342B34202F2032202D203823
:10064000202F2033202D20382B34202F2034202D14
:10065000203132202F2035202D2031322B34202FF5
:100660002036202D20313600536574204368616E9A
:100670006E656C20636F6E6669673A20005365741F
:100680002044617461726174652028302D32293AEA
:10069000200053657420486F70206368616E6E653A
:1006A0006C7320286D61782032342C207365706162
:1006B000726174656420627920636F6D6D61732966
:1006C0002076616C69642076616C75657320312DCC
:1006D0003235353A2000536574206368616E6E656B
:1006E0006C2073706163696E6720287831306B48C5
:1006F0007A293A200053657420524620706F77653E
:10070000722028302D37293A200053657420524634
:10071000206D6167696320286865782920652E67E8
:100720002E20307844454144463030443A2000532E
:1007300065742062617365206672657175656E63AC
:10074000792028696E20487A293A20005B5A5D207A
:10075000656E746572207265636569766572206383
:100760006F6E66696775726174696F6E2075746902
:100770006C79005B465D20646973706C61792061FF
:10078000637475616C206672657175656E63696509
:10079000732075736564005B525D2063616C6375E3
:1007A0006C6174652072616E646F6D206B65792079
:1007B000616E6420686F70206C697374005B495DC2
:1007C000207265696E697469616C697A6520736508
:1007D0007474696E677320746F20736B65746368DB
:1007E0002064656661756C7473005B585D2072658A
:1007F00076657274206368616E67657320616E64EC
:100800002065786974206D656E75005B535D20739B
:100810006176652073657474696E677320746F20E8
:10082000454550524F4D20616E64206578697420B3
:100830006D656E7500557365206E756D62657273BA
:10084000205B302D395D20746F20656469742070E1
:100850006172616D657465727300202D2053797328
:1008600074656D20636F6E66696775726174696F18
:100870006E000A0A6F70656E4C52536E672000510D
:1008800029204F7574707574206265666F726520DB
:100890006C696E6B20283D465329203A2000502970
:1008A00020536C617665206D6F64652028657870D3
:1008B0006572696D656E74616C293A20004F29205C
:1008C00054696D65642042494E44206174207374FC
:1008D000617274757020203A20004E292050504DCE
:1008E000206F7574707574206C696D69746564200F
:1008F000202020203A200044495341424C454400E6
:100900004D292050504D205253534920746F20637D
:1009100068616E6E656C202020203A20004C2920F2
:1009200050504D206D696E696D756D2073796E63E1
:10093000202875732920203A200044495341424C15
:100940004544004B29204661696C736166652062ED
:100950006561636F6E20696E74762E2028312D32AA
:10096000353573293A20004A29204661696C736144
:10097000666520626561636F6E2064656C617920D5
:1009800028302D323535203D3E20313073202D204A
:100990003135306D696E293A200049292046616958
:1009A0006C7361666520626561636F6E206672714B
:1009B0002E203A200048292050574D2073746F7024
:1009C0002064656C6179202020202020203A2000BE
:1009D00047292050504D2073746F702064656C61FE
:1009E00079202020202020203A200046292046611E
:1009F000696C736166652064656C617920202020D4
:100A00002020203A200050574D206368616E6E65AB
:100A10006C200066756E6374696F6E3A2000292041
:100A2000706F72742000506F776572546F776572C3
:100A300000445446205548462033322D62697420C4
:100A400031306368004F70656E4C52536E67525878
:100A5000206D696E6920342F36636800466C7974A6
:100A6000726F6E2F4F72616E6765525820554846FF
:100A70002038636800525820747970653A20004429
:100A8000697361626C656400487A00203D3D200016
:100A900043616C63756C61746564207061636B6540
:100AA0007420696E74657276616C3A200042292068
:100AB0004D6963726F202868616C66292050504D23
:100AC000202020203A00412920496E766572746505
:100AD000642050504D20696E20202020203A0030A4
:100AE00029204D7574652062757A7A657220286DAB
:100AF0006F73746C79293A003929205365726961E2
:100B00006C2062617564726174653A00736D617224
:100B100074506F7274004672536B79005472616E38
:100B200073706172656E740044697361626C6564B0
:100B30000038292054656C656D657472793A2020FF
:100B40002020202020003729204368616E6E656CCC
:100B500020636F6E6669673A202000362920446161
:100B60007461726174652028302D32293A2020206A
:100B700000352920486F70206368616E6E656C7364
:100B80003A2020202020003429204368616E6E65C1
:100B90006C2073706163696E673A202000332920EE
:100BA000524620706F7765722028302D37293A2001
:100BB0002020003229205246206D616769633A2067
:100BC0002020202020202020003129204261736530
:100BD000206672657175656E63793A202020000089
:100BE00000000700020100000304060000000000EE
:100BF00000000001020408102040800102040810D7
:100C00002001020408102004040404040404040263
:100C10000202020202030303030303000000002395
:100C2000002600290000000000250028002B0000FD
:100C3000000000240027002A0000E82D11241FBE18
:100C4000CFEFD8E0DEBFCDBF13E0A0E0B1E0EEED26
:100C5000F1E602C005900D92A83CB107D9F716E065
:100C6000A8ECB3E001C01D92A239B107E1F71CE086
:100C7000CCE3DCE004C02297FE010E94F12ECA33CF
:100C8000D107C9F70E94242E0C94ED300C9400007B
:100C900080917705813019F482E080937705809107
:100CA0007705833019F484E0809377050895A8953B
:100CB0000895DC01ED91FC910190F081E02D099502
:100CC00008952091780530917905382748E0C901C9
:100CD000880F991F37FF06C09C0151E2252750E17C
:100CE000352701C09C01415091F73093790520933D
:100CF0007805089588E380937A0580E092ECA1E07E
:100D0000B0E080937B0590937C05A0937D05B09324
:100D10007E0587E08093870580EC92E9ADEEB9E12E
:100D200080937F0590938005A0938105B093820501
:100D300085E0809388058DEE9EEFADEABEED809351
:100D4000830590938405A0938505B0938605E9E813
:100D5000F5E080E090E0863028F4DC01AE54BC4F32
:100D60002C9101C020E0219301968831910599F7DB
:100D700082E08093A1058AE08093A205089580EC2B
:100D800091EDA8E9BBE18093BF059093C005A093C6
:100D9000C105B093C20580E090E0A0E0B0E580938B
:100DA000C3059093C405A093C505B093C605E7ECB1
:100DB000F5E080E081938F5F8031E1F70895A0E056
:100DC000B0E0E5EEF6E00C94BA2ED82F0E941F2971
:100DD0006115710581059105C9F30E945D2F10927F
:100DE0008305109284051092850510928605C4E053
:100DF000812C912C54018A94C0908305D090840555
:100E0000E0908505F0908605FE2CED2CDC2CCC24A2
:100E10000E94582FA50194010E94992E6C0D7D1DF2
:100E20008E1D9F1D609383057093840580938505B7
:100E300090938605C15001F7DD2309F450C009E8FD
:100E400015E0E801A12CB12C62E3C62ED12CE12CD7
:100E5000F12C8881882309F442C0B39419F40E94CC
:100E60007A063DC00E94582FA70196010E94992E34
:100E7000E1E0E60FA9E8B5E08A2F801B8A1520F48F
:100E80008D918E13F9CFE9CF2091880530E0A0E154
:100E9000B7E20E94312E9B01AC01AE2FB0E00E9460
:100EA000402E40907F0550908005609081057090A5
:100EB0008205640D751D861D971D4090BF055090DD
:100EC000C0056090C1057090C205461657066806B9
:100ED000790618F2E993A39488E1A812BACFCDB7A6
:100EE000DEB7E0E10C94D62E8436910520F4BC01E7
:100EF00080E090E017C09C018E3B910528F42A55B4
:100F00003109AAE0B0E00CC0823D910528F4245BD1
:100F10003109A4E6B0E004C02D5C3109A8E5B2E0D7
:100F20000E94312EA4E6B0E09B01AC010E94402E4D
:100F3000089590E08C599F4F0E947407089561E0D6
:100F400083E10E94CC2960E083E10E94052A82E0CF
:100F50008093B00085E08093B10061E083E00E945F
:100F6000CC2960E083E00E94052A0895A4E0B0E067
:100F7000ECEBF7E00C94C82E009749F19C0140E09F
:100F800050E068E478EE81E090E00E94992E61E004
:100F900083E129833A834B835C830E94052A29815C
:100FA000822F3A81932F4B81A42F5C81B52F8F3FE5
:100FB0009105A105B10529F020F08FEF90E0A0E0A8
:100FC000B0E08093B3008091B000806107C060E022
:100FD00083E10E94052A8091B0008F7E8093B0004B
:100FE0002496E2E00C94E42E60E08CE00E94CC2990
:100FF00061E08BE00E94CC2961E08DE00E94CC2969
:1010000060E082E00E94CC2961E084E00E94CC296B
:10101000089542E050E068E476E080E00E944F28C6
:101020000895E3E0F0E089E080935700E491E670F2
:1010300081E0E63009F080E00895CF93DF93C82F78
:101040000E941108882381F0DFB781E08093760544
:10105000F8940E94570688E180936000C093600076
:10106000C1110E945706DFBFDF91CF9108958F9283
:101070009F92AF92BF92CF92DF92EF92FF92CF9367
:10108000FC01C0A5EC2FE770F0E0E658FC4FA08112
:10109000B0E0C7FF03C024E130E002C02FE030E041
:1010A000FC0197A183E1989FF0011124E25CFE4FBF
:1010B00080809180A280B380A20FB31F20E43FE123
:1010C0004DE750E00E944B2EA50194010E94772E1F
:1010D0008C2F887149F469017A01E0EDCE0EE7E0CA
:1010E000DE1EE11CF11C1BC0C7FF05C060E47AE8EE
:1010F0008CE29EE004C060E07EEE8AEB9BE069013A
:101100007A01F8EBCF0EFBE0DF1EE11CF11CA5011C
:1011100094010E94772EC20ED31EE41EF51EC70155
:10112000B60169517C4F8F4F9F4F28EE33E040E06E
:1011300050E00E94772EA8EEB3E00E94402ECF919F
:10114000FF90EF90DF90CF90BF90AF909F908F90E7
:1011500008958F3F910551F048F0811522E09207E4
:1011600038F08115934030F482E0089580E00895CE
:1011700081E0089583E00895A0E0B0E0E2ECF8E0BB
:101180000C94C32EEB018A01B82FB695A0E02881FC
:101190003981F80120832A813B8121832C813D8183
:1011A00022832E813F812383688179814A815B81FB
:1011B0002C813D81EE81FF819F2F9295990F990F90
:1011C000907C272F2370922B252F2370220F220F24
:1011D000922B232F23702295207F922BF80194834A
:1011E0000B5F1F4F2896AF5FBA1788F680FF24C0A9
:1011F000888199810E94A908D82E8A819B810E94AA
:10120000A908E82E8C819D810E94A908F82E8E8164
:101210009F810E94A908F0E4DF9EA001112490E1C3
:10122000E99E90011124242B282BE4E0FE9EB001BE
:101230001124262BF8012083CDB7DEB7E7E00C940C
:10124000DF2E803223E0920708F1883E23E09207E8
:1012500040F48F519340E4E096958795EA95E1F745
:101260000895803D27E0920718F48C5D934008951F
:10127000883928E0920768F4885C974074E0969576
:1012800087957A95E1F78D509C4F089580E090E026
:1012900008958FEF93E008958C30910540F4A4E019
:1012A000880F991FAA95E1F7885D9C4F0895843FA8
:1012B00023E0920718F484529C4F0895811524E08E
:1012C000920740F48657934FF4E0880F991FFA95E0
:1012D000E1F7089580E998E008959C0136952795F7
:1012E00025753575821B930B9C012373337396957B
:1012F00087959695879583739373820F931F9C01AF
:1013000054E0369527955A95E1F7280F391F2F702D
:101310003F7041E051E0249FC001259F900D349F14
:10132000900D1124892F08952D98882319F000001D
:101330002B9A02C000002B9800002D9A00000895FF
:101340002D9A000083B12D98000082958170089538
:10135000CF93DF93D82F5C9A2D985C98C8E08D2F9F
:1013600080780E949409DD0FC150C9F72D98DF9154
:10137000CF9108958F770E94A8090895CF93DF93A6
:10138000D82FC8E08D2F80780E949409DD0FC150BE
:10139000C9F72D98DF91CF910895CF93DF932D98C2
:1013A000C8E080E0D82FDD0F0E94A0098D0FC1504A
:1013B000C9F7DF91CF9108950E94BA090E94CD0923
:1013C0005C9A0895A1E0B0E0E8EEF9E00C94C82E34
:1013D000806869830E94A8096981862F0E94BE09DE
:1013E0005C9A2196E2E00C94E42ECF93C0918305A1
:1013F000C827E82FF0E0E658FA4F678589E70E9492
:10140000E2096C2F8DE30E94E2096C2F82E40E94B6
:10141000E209CF91089586E20E94DC090895CF93F6
:10142000DF93EC016C818CE10E94E2096D818DE11A
:101430000E94E2096E818EE10E94E2096F8180E2E2
:101440000E94E209688581E20E94E209698582E2E0
:101450000E94E2096A8583E20E94E2096B8584E2C8
:101460000E94E2096C8585E20E94E2096D858AE2AC
:101470000E94E2096E858EE60E94E2096F858FE682
:101480000E94E209688980E70E94E209698981E790
:101490000E94E2096A8982E70E94E209DF91CF9106
:1014A0000895CF92DF92EF92FF92CF93DF936B017B
:1014B0007C01C11488E3D8068CE9E8068CE1F806C3
:1014C00028F5C701B60120E836E948E950E00E9456
:1014D000772EE901689760E879E687E69FEF0E943A
:1014E000532E6C0D7D1D8E1D9F1DF2E0660F771F24
:1014F000881F991FFA95D1F721E732E040E050E0CC
:101500000E94772EF22EE32E80E421C0C701B6019F
:1015100020E03DE241E351E00E94772EE901689727
:1015200060E073ED8EEC9EEF0E94532E6C0D7D1DDE
:101530008E1D9F1D660F771F881F991F21E732E0C0
:1015400040E050E00E94772EF22EE32E80E66C2FD2
:101550006F71680F85E70E94E2096E2D86E70E9491
:10156000E2096F2D87E70E94E209DF91CF91FF909A
:10157000EF90DF90CF900895682F8DE60E94E209EA
:1015800008958F929F92AF92BF92CF92DF92EF9287
:10159000FF92CF93DF93D82F83E00E94DC098093E2
:1015A000750584E00E94DC098093740560E086E0A4
:1015B0000E94E20961E087E00E94E2096FE789E0AA
:1015C0000E94E20965E08AE00E94E20962E18BE0A4
:1015D0000E94E20965E18CE00E94E2096DEF8DE076
:1015E0000E94E20960E08EE00E94E209DD2319F02A
:1015F0008BE291E008C02091A10533E1239FC00157
:101600001124825C9E4F0E940F0A6CE880E30E94C6
:10161000E2096FE082E30E94E20962E483E30E9450
:10162000E2098091A20587FF02C064E101C06AE07F
:1016300084E30E94E2096AE285E30E94E2096DE226
:1016400086E30E94E20964ED87E30E94E20960E01C
:1016500088E30E94E20960E089E30E94E209D11177
:1016600009C0C0908305D0908405E0908505F09076
:10167000860507C0C5E9CC2EC1ECDC2EED2CCEEDE5
:10168000FC2ECAE38F2C9924AA24BB24682D8C2F0E
:101690000E94E209682D85E08C0F0E94E209FE2C71
:1016A000ED2CDC2CCC24CF5FCE3361F76FEF83E4DD
:1016B0000E94E2096FEF84E40E94E2096FEF85E483
:1016C0000E94E2096FEF86E40E94E209DD2311F037
:1016D00066E002C0609187058DE60E94E20960E045
:1016E00089E70E94E209609188058AE70E94E20981
:1016F00060E083E70E94E20960E084E70E94E2097B
:10170000D11109C060917F0570918005809181059C
:101710009091820504C060EC72E98DEE99E10E941F
:10172000510ADF91CF91FF90EF90DF90CF90BF9063
:10173000AF909F908F90089561E087E00E94E2094A
:1017400064E28EE70E94E20963E088E00E94E20919
:1017500060E088E00E94E20965E087E00E94E2091B
:1017600062E085E00E94E20983E00E94DC09809348
:10177000750584E00E94DC0980937405089583E078
:101780000E94DC098093750584E00E94DC09809347
:10179000740561E087E00E94E2096AE070E080E0A1
:1017A00090E00E9442290E949C0B00000895CF9275
:1017B000DF92FF920F931F93CF93DF931F92CDB7CA
:1017C000DEB7082F162F8EE399830E94E209F02ED0
:1017D000C02E9981D92E8C2D8F19811738F4F601DE
:1017E00061916F018FE70E94E209F5CF64E085E027
:1017F0000E94E20983E00E94DC098093750584E081
:101800000E94DC09809374050E941F296093700573
:1018100070937105809372059093730569E087E07A
:101820000E94E20981E0809377050F90DF91CF91CC
:101830001F910F91FF90DF90CF9008950F931F930A
:101840000E94D70B80917705813099F40E941F295F
:10185000009170051091710520917205309173050A
:10186000601B710B820B930B603A764881409105A7
:1018700048F380917705813031F46EE971E086EEAE
:1018800095E00E940B2B1F910F9108950F931F93CA
:1018900080917705823021F41092770581E020C095
:1018A000809177058130D9F40E941F29009170053D
:1018B000109171052091720530917305601B710BB9
:1018C000820B930B613A76488140910540F061E0CC
:1018D00087E00E94E2091092770582E001C080E073
:1018E0001F910F910895CF93DF93EC014AE050E0F0
:1018F0006D2F70E086EE95E00E94D92B6EE286EEA9
:1019000095E00E94DD2ABE0184E0769567958A9570
:10191000E1F76F7077274AE050E086EE95E00E948D
:10192000D92B6EE286EE95E00E94DD2ABE016F7033
:1019300077274AE050E086EE95E00E94D92BDF91B0
:10194000CF910895D82FC0E0CD1790F45E9A409AB9
:1019500064E670E080E090E00E9442295E98409842
:1019600064E670E080E090E00E944229CF5FECCF17
:101970006CE271E080E090E00E944229E4CF0F9396
:101980001F93CF93DF93EC01062F15E0115051F018
:10199000CE010E94D430081741F0602FCE010E9482
:1019A000DC30F4CF82E00E94A20CDF91CF911F9136
:1019B0000F910895A0E0B0E0E0EEFCE00C94BA2EA8
:1019C000482E562EC0E0D0E0612C712CE12CF12C79
:1019D00000E010E041100CC06090D80586E4689EDD
:1019E0003001112459E1E52EF12C0EEB15E01EC05B
:1019F00091E049120FC06090D805E6E46E9E300178
:101A00001124FBE16F0E711C49E2E42EF12C0AE770
:101A100015E00CC082E0481209C028E1622E77244C
:101A20007394EE24E394F12C07ED15E043018C0E42
:101A30009D1E10927905109278053401A62CA818E5
:101A4000B12CC30101966C01AE14BF04A8F4A00E22
:101A5000B11E511006C0C3010E94D430F50180832D
:101A600005C0F5016081C3010E94BF0CF5018081B2
:101A70000E9461063601E2CFC301511018C0C301B4
:101A80000E94D430B82EC6010E94D4302B2D30E0F5
:101A9000322F2227282B8091780590917905821783
:101AA000930779F4C0E0D0E05524539493CF3601E6
:101AB000609179050E94BF0C60917805C6010E9473
:101AC000BF0CC05EDE4FC13E92E0D90708F482CF62
:101AD000852DCDB7DEB7E0E10C94D62E61E082E033
:101AE0000E94DA0C089560E082E00E94DA0C809196
:101AF000D705853020F01092D7050E946E0D809199
:101B0000D7058093D805089561E080E00E94DA0C43
:101B100061E081E00E94DA0C089560E080E00E94BC
:101B2000DA0C882351F060E081E00E94DA0C88230F
:101B300021F080917A05883349F00E94BF060E9407
:101B40007A0681E00E94DF060E94840D08958823B2
:101B500019F06AEA71E002C06EEA71E086EE95E083
:101B60000E940B2B0895FF920F931F93CF93DF9347
:101B700069EC7BE086EE95E00E94B72A40917F05F4
:101B80005091800560918105709182052AE030E0D6
:101B900086EE95E00E94E02B63EB7BE086EE95E01D
:101BA0000E94B72A40918305509184056091850574
:101BB0007091860520E130E086EE95E00E94E02BF2
:101BC0006DE97BE086EE95E00E94B72A4AE050E09E
:101BD0006091870586EE95E00E94082C67E87BE01F
:101BE00086EE95E00E94B72A4AE050E060918805B1
:101BF00086EE95E00E94082C61E77BE086EE95E09A
:101C00000E94B72AC9E8D5E0F12C8E01888188238B
:101C1000A9F0FF2031F061EB71E086EE95E00E94C3
:101C2000DA2A21964AE050E0F801608186EE95E0DC
:101C30000E94D12BF394F8E1FF12E7CF86EE95E0F6
:101C40000E94E52A6BE57BE086EE95E00E94B72ACC
:101C50004AE050E06091A10586EE95E00E94082CD4
:101C600066E47BE086EE95E00E94B72AE091A2054B
:101C7000E770F0E0EE0FFF1FEE57FC4F60817181BF
:101C800086EE95E00E940B2B61E37BE086EE95E00B
:101C90000E94B72A8091A2058871883069F028F4E3
:101CA000811113C068E27BE00CC0803141F08831C3
:101CB00061F46CE07BE005C06CE17BE002C066E1B2
:101CC0007BE086EE95E00E94F92A68EF7AE086EEE6
:101CD00095E00E94B72A40917B0550917C05609168
:101CE0007D0570917E052AE030E086EE95E00E9449
:101CF000E02B6FED7AE086EE95E00E94B72A8091A6
:101D0000C30580710E94A70D66EC7AE086EE95E02F
:101D10000E94B72A8091C30580740E94A70D6DEAC6
:101D20007AE086EE95E00E94B72A8091C305807222
:101D30000E94A70D60E97AE086EE95E00E94B72A3E
:101D40008AE795E00E943708AB01BC012AE030E049
:101D500086EE95E00E94C22B6BE87AE086EE95E075
:101D60000E94B72A8AE795E00E9437089B01AC01E0
:101D700060E472E48FE090E00E94772EBA01A9013E
:101D80002AE030E086EE95E00E94C22B68E87AE017
:101D900086EE95E00E94F92ACDB7DEB7E5E00C9417
:101DA000E12E8F929F92AF92BF92CF92DF92EF92ED
:101DB000FF92811107C06FE77AE086EE95E00E94FE
:101DC000F92A2FC090E00E94740724E630E040E03A
:101DD00050E00E94772ECA01B9012AE030E040E0CD
:101DE00050E00E94772E49015A016B017C012AE0E4
:101DF00030E0B501A40186EE95E00E94C22B6EE2B0
:101E000086EE95E00E94DD2A2AE030E0B701A601C7
:101E100086EE95E00E94C22B63E786EE95E00E9475
:101E20001D2BFF90EF90DF90CF90BF90AF909F90D1
:101E30008F9008951F93CF93DF9365E77AE086EE46
:101E400095E00E94B72A8091A305813041F46CE5AA
:101E50007AE086EE95E00E94F92A10E050C08230C8
:101E600019F465E47AE0F5CF843019F461E37AE09F
:101E7000F0CF853091F766E27AE0EBCFC12FD0E06A
:101E8000C930D1050CF441C068E3610F86EE95E0DE
:101E90000E94DD2A6EE17AE086EE95E00E94B72A84
:101EA000BE016F5F7F4F4AE050E086EE95E00E94F2
:101EB000A12B63E17AE086EE95E00E94B72ACD552A
:101EC000DA4FE981E03218F566E07AE086EE95E0D7
:101ED0000E94B72A8981803130F06DE673E086EE8A
:101EE00095E00E94DA2A69816F7070E06F5F7F4F22
:101EF0004AE050E086EE95E00E94AA2B1F5F809199
:101F00004C05181708F4BACF0FC061E3BECFEF70CD
:101F1000F0E0EE0FFF1FEE56FC4F6081718186EE00
:101F200095E00E940B2BEACF6BEE79E086EE95E010
:101F30000E94B72A8091BB050E94D10E60ED79E026
:101F400086EE95E00E94B72A8091BC050E94D10ED2
:101F500065EB79E086EE95E00E94B72A8091BD0599
:101F60000E94D10E6AE979E086EE95E00E94B72AD8
:101F70004091B3055091B4056091B5057091B605D7
:101F8000411551056105710539F12AE030E086EE11
:101F900095E00E94E02B67E679E086EE95E00E94EE
:101FA000B72A8091B7050E949907AB01BC012AE0CE
:101FB00030E086EE95E00E94E02B63E479E086EE67
:101FC00095E00E94B72A4AE050E06091B80586EE9D
:101FD00095E00E94082C06C06AE379E086EE95E061
:101FE0000E94F92A6DE179E086EE95E00E94B72A19
:101FF0006091B9057091BA054AE050E086EE95E02F
:102000000E94F22B60E079E086EE95E00E94B72A0C
:102010006091B205603450F470E06F5F7F4F4AE02A
:1020200050E086EE95E00E94AA2B06C067EF78E0AC
:1020300086EE95E00E94F92A6AED78E086EE95E05A
:102040000E94B72A8091B10580FF03C063EB71E065
:1020500002C067EB71E086EE95E00E940B2B6DEB02
:1020600078E086EE95E00E94B72A8091B1058270F3
:102070000E94A70D6EE978E086EE95E00E94B72AEF
:102080008091B10584700E94A70D6FE778E086EE1D
:1020900095E00E94B72A8091B10588700E94A70D33
:1020A000DF91CF911F9108950F931F93CF93DF93EB
:1020B000209149052F3FA9F56FEF75E086EE95E079
:1020C0000E94B72A88E893E00E94730C6EED75E0D9
:1020D00086EE95E00E94B72A80914A0590914B05C3
:1020E0000E94730C6BEA75E086EE95E00E94F92A77
:1020F00068E875E086EE95E00E94F92A60E775E0F1
:1021000086EE95E00E94F92A6BE475E086EE95E094
:102110000E94F92A86EE95E00E94E52A0E941A0F95
:1021200068C012160CF065C0332727FD30958091EA
:102130004C0590E0821793070CF45BC066E375E0F2
:1021400086EE95E00E94B72A60914905772767FDE2
:1021500070954AE050E086EE95E00E94AA2B6BE075
:1021600075E086EE95E00E94B72A10E008E28091C3
:102170004D051817D0F5C12FD0E0CC0FDD1FC25B85
:10218000DA4F288130E080914905992787FD9095A5
:1021900001972817390739F56BEB71E086EE95E06A
:1021A0000E94DA2A4AE050E0602F86EE95E00E9415
:1021B000D12B6FEB71E086EE95E00E94DA2AE9817F
:1021C000EF70F0E0EE0FFF1FEE56FC4F6081718163
:1021D00086EE95E00E94DA2A63EC71E086EE95E0E7
:1021E0000E94DA2A0F5F1F5FC2CF86EE95E00E9441
:1021F000E52ADF91CF911F910F910895FF920F93E0
:102200001F93CF93DF93C9E8D5E0F12C8E0188812D
:102210008823D1F165EC71E086EE95E00E94DA2A20
:102220004AE050E06F2D86EE95E00E94D12B62EDE2
:1022300071E086EE95E00E94DA2A2196F80120816D
:1022400030E0A0E1B7E20E94312E9B01AC01A091E9
:102250008805B0E00E94402EAB01BC0180917F0553
:1022600090918005A0918105B0918205480F591F7A
:102270006A1F7B1F2AE030E086EE95E00E94E02B8B
:10228000F394F8E1FF12C2CFCDB7DEB7E5E00C94CE
:10229000E12E1092E30485E6E4EEF4E0DF011D9206
:1022A0008A95E9F70895CF93C82F8F3719F08830B2
:1022B00009F045C0E091E304EE23D9F1E150E09349
:1022C000E304F0E0EC51FB4F10826DE070E086EE2D
:1022D00095E00E945906C0E08091E304C81760F4BD
:1022E000EC2FF0E0EC51FB4F608170E086EE95E062
:1022F0000E945906CF5FF0CF60E270E086EE95E075
:102300000E9459066DE070E086EE95E00E94590645
:10231000C0E08091E304C81778F5EC2FF0E0EC51B1
:10232000FB4F608170E086EE95E00E945906CF5F1A
:10233000F0CF67E086EE95E00E94DD2A1DC08B316C
:1023400019F40E9449111AC08D30C1F08A30B1F0E1
:102350008091E304843668F76C2F70E086EE95E098
:102360000E945906E091E30481E08E0F8093E3041C
:10237000F0E0EC51FB4FC08380E001C081E0CF91E1
:102380000895CF93C82F0E941F296093CC047093A7
:10239000CD048093CE049093CF04C093E104CC236A
:1023A00029F040E051EE60E070E004C040E855E202
:1023B00060E070E086EE95E00E94672DCF91089571
:1023C0009091D004492F4F7050E0BA016F5F7F4F5A
:1023D000292F30E0E4E035952795EA95E1F762177B
:1023E000730759F0FA01EF52FB4F808381E0890FA8
:1023F0008F70907F892B8093D00408956EE770E0F2
:1024000086EE95E00E9459060895A3E1B1E0EBE065
:10241000F2E10C94BB2EE9E8F5E0712C8191882360
:1024200021F0739428E17212F9CF66ED71E086EE27
:1024300095E00E940B2B4AE050E0672D86EE95E078
:102440000E94082C80E00E94C10A0E949C0B8E0111
:102450000E5F1F4FC12CD12C7601C39466246A9461
:102460005C2C0E9413294B015C012091880530E00F
:10247000A0E1B7E20E94312E9B01AC01C701B60179
:102480000E94532E20917F05309180054091810557
:1024900050918205620F731F841F951F2091BF0505
:1024A0003091C0054091C1055091C20526173707EC
:1024B0004807590718F4F801608229C08C2D0E9442
:1024C000F50961E070E080E090E00E944229F801A7
:1024D00010820E941329681979098A099B09643FAF
:1024E00071408105910540F40E940B0AF80190812A
:1024F000981778F78083EDCF50FE05C05D9841981E
:102500005E9A409A04C05D9A419A5E9840982FEF77
:10251000C21AD20AE20AF20A0F5F1F4F8FEFC816E3
:10252000D104E104F10409F09BCFCE019395FC01A5
:10253000D82E7FEF68EC2E2F281B271510F051E0C6
:1025400056C0DE01129651E02FEF41E03D91321767
:1025500010F0322F01C0452F5F5F5F3F11F0232F36
:10256000F5CF4193242F30E0A1E0B0E0AC0FBD1FC8
:10257000A20FB31F5C93413079F0DE01A20FB31FAD
:102580005C93423049F0AFEFBFEFAC0FBD1FA20F1D
:10259000B31F6C934E3F78F6A2E0B0E0AC0FBD1FC6
:1025A000A20FB31F7C934D3F30F6A3E0B0E0AC0F19
:1025B000BD1FA20FB31F6C93BECF452F242F30E059
:1025C000FC01E20FF31F6081AFEFB0E0AC0FBD1F65
:1025D000A20FB31F2C91621748F44150DC01A40FE5
:1025E000B11D2C9120836C934111E8CF5F5F57158B
:1025F00020F3372D369520E0231770F4DC01A20F6D
:10260000B11D4C91522F530FFC01E50FF11D50816C
:102610005C9340832E5FF0CFF9E8EF2EF5E0FF2EBC
:102620008C01802F8D19871598F4F801C1908F01C6
:102630004AE050E06C2D86EE95E00E94D12B6CE2D2
:1026400086EE95E00E94DD2AF701C1927F01E9CF75
:1026500086EE95E00E94E52A81E0CD5EDE4FEFE058
:102660000C94D72E1F920F920FB60F9211241F9326
:102670002F933F934F935F936F937F938F939F938A
:10268000AF93BF93CF93DF93EF93FF93C0918600F7
:10269000D091870080918704909188042091A904AB
:1026A000211155C09E01281B390B8091C3059091C3
:1026B000C405A091C505B091C60585FD02C036953B
:1026C0002795253C49E03407B8F140910A0150E0D4
:1026D00060E070E02CE1B695A795979587952A95CF
:1026E000D1F70097A105B10521F481E090E0A0E0C9
:1026F000B0E084179507A607B707D8F480910A01C0
:102700008F3FB9F040E080910A01481780F4842F90
:1027100090E0880F991FFC01E757FB4F2081318122
:10272000FC01E55FFE4F318320834F5FECCF1092B9
:10273000AA0410920A010BC02D3B82E0380720F05A
:1027400080910A018031D8F08FEF80930A01D093F5
:102750008804C0938704FF91EF91DF91CF91BF91DF
:10276000AF919F918F917F916F915F914F913F9129
:102770002F911F910F900FBE0F901F9018951091E1
:102780000A0181E0810F80930A01C9010E94210999
:10279000E12FF0E0EE0FFF1FE757FB4F918380839F
:1027A000D6CF83E0809380008AE980938100809176
:1027B000C30586FD05C080918100806480938100FF
:1027C0008FEF9FEF909389008093880080916F0036
:1027D000806280936F0008950E94730D8091D805E8
:1027E000843011F41092D80508956F3018F0869552
:1027F0008058089589E0689F802D11240895A0E0F5
:10280000B0E0E5E0F4E10C94C22EC82F0E941F292D
:10281000009138041091390420913A0430913B041E
:102820006B017C01C01AD10AE20AF30A9701860102
:1028300049E8C41643E1D406E104F10410F0109213
:102840003C04609338047093390480933A04909365
:102850003B042091A9048FEF820F8230E8F5E091CC
:102860003C04EE2309F46EC1E13011F482E0D8C1DA
:10287000E03178F581E08E0F80933C04F0E0E7577B
:10288000FB4FC083803109F0D4C1EBE8F4E0213084
:1028900029F4A181A695A695808108C080819181A7
:1028A000A92FA695A695A69596958795A03148F44B
:1028B000B0E090E0AA0FBB1FA55FBE4F11969C939E
:1028C0008E931092AA04329684E0E939F807F9F65B
:1028D000B0C110923C04ADC1233009F023C1E09196
:1028E0003C04E11118C0CF3009F011C10E94132936
:1028F0000091B7041091B8042091B9043091BA0442
:10290000601B710B820B930B623071058105910581
:1029100008F089C1FCC0E73148F481E08E0F809354
:102920003C04F0E0E857FB4FC083F1C0E73109F009
:10293000ECC0C111EAC040E050E0ABE0CA01B3E036
:10294000880F991FBA95E1F7A49F9001A59F300DBC
:102950001124F901E757FB4F6081E1817E2F7770E9
:1029600075956795FC01EE0FFF1FE55FFE4F7183C4
:102970006083F901E657FB4FB081B695B695B695E1
:10298000E181FE2FF295FF0FF07E6F2F6B2BE69506
:10299000E695E6957E2F777075956795FC01EE0FAD
:1029A000FF1FE35FFE4F71836083F901E557FB4F23
:1029B000B081B295B695B695B370C181DC2FDD0FAD
:1029C000DD0F6D2F6B2BC295C695C695C370E28146
:1029D000E170EE0FEE0F7E2F7C2B75956795FC0155
:1029E000EE0FFF1FE15FFE4F71836083F901E35734
:1029F000FB4FB081B695E181FE2FF795FF27F79544
:102A00006F2F6B2BE6957E2F777075956795FC0180
:102A1000EE0FFF1FEF5EFE4F71836083F901E257F7
:102A2000FB4FB081B295BF70E181FE2FF295F07F30
:102A30006F2F6B2BE295EF707E2F777075956795F2
:102A4000FC01EE0FFF1FED5EFE4F71836083F90105
:102A5000E157FB4FB081BB1FBB27BB1FC181DC2FE0
:102A6000DD0F6D2F6B2BCC1FCC27CC1FE281E370C9
:102A7000EE0F7E2F7C2B75956795FC01EE0FFF1FE7
:102A8000EB5EFE4F71836083F901EF56FB4FB0811F
:102A9000B695B695E181FE2FF295FF0FFF0FF07C02
:102AA0006F2F6B2BE695E6957E2F77707595679562
:102AB000FC01EE0FFF1FE95EFE4F71836083F90199
:102AC000EE56FB4F20812295269527703181E32F0A
:102AD000EE0FEE0FEE0F6E2F622B732F7295769521
:102AE000777075956795FC01EE0FFF1FE75EFE4F4F
:102AF000718360834F5F5F4F4230510509F01ECFF5
:102B000080919F0483FF1092AA0410923C040E94BB
:102B100013296093B7047093B8048093B904909319
:102B2000BA0487C0243009F084C060913C0461116C
:102B30000BC0C83AB1F4109279051092780588EA72
:102B40000E94610681E06CC0613019F4C0933704C3
:102B500004C0623031F4C09336048C2F0E946106A9
:102B60005AC0E09136042E2F30E0220F331F462F3B
:102B700050E0C9010296841795073CF0633268F76C
:102B8000FA01EA57FB4FC083E8CF2D5F3F4F8C2FF0
:102B900090E060917805709179054217530749F4E8
:102BA000982F882786279727909379058093780513
:102BB00032C06817790769F580913704813049F58B
:102BC000E13118F080E180933604F0903604CAE8D1
:102BD000D4E000E010E00F15D0F4FE0131978081C1
:102BE00090E0982F88272881822B63E0969587951F
:102BF0006A95E1F70E942109F801EE0FFF1FE55FDA
:102C0000FE4F918380830F5F1F4F2296E4CF109277
:102C1000AA0410923C0480913C04882351F08F5FF9
:102C200080933C0406C080913C048F5F80933C04F9
:102C30006ECFCDB7DEB7E8E00C94DE2EE82FF0E0E3
:102C4000E254FA4FE185E03150F4F894F0E0EE0FF1
:102C5000FF1FE55FFE4F80819181789408958EE09B
:102C60008E0F8B3058F4F0E0E25FF10924E62E9FDE
:102C7000C0012F9F900D11240C960895E03FF1F0B4
:102C800028F4E03161F0E13161F006C0ED3F81F000
:102C9000EE3F89F0E13F49F080E092E0089582E163
:102CA00001C083E10E94612A089586E090E00895C2
:102CB0008AEF93E008958FEF93E0089580E090E02D
:102CC0000895A2E2B0E0E7E6F6E10C94B82E9E018A
:102CD0002F5F3F4F80E1D9011D928A95E9F764E0AB
:102CE00072E086EE95E029A33AA30E940B2B0E9486
:102CF000BF0B1D8A1E8A1F8A188E312C212C00E0E2
:102D0000812C912C540170E4472E71EE572E7DE9F1
:102D1000672E78E1772EE0E5CE2EE3ECDE2EE12C77
:102D2000F12C84EF91E0A0E0B0E08D8F9E8FAF8F0B
:102D3000B8A380EC91EDA8E9BBE1898F9A8FAB8FA6
:102D4000BC8F80E491EEADE9B8E1898B9A8BAB8BB7
:102D5000BC8B86EE95E00E941F2C892B09F4E1C004
:102D600086EE95E00E944C2C9C0133272C323105D5
:102D700009F442C0ACF42332310509F0ABC019822A
:102D80001A821B821C821D821E821F82188619864F
:102D90001A861B861C861D861E861F86188A60C0A2
:102DA0002434310529F02335310509F4B2C092C02D
:102DB00064E486EE95E00E94DD2A2AE030E040E4FB
:102DC00051EE6DE978E186EE95E00E946B2B6CE2A6
:102DD00086EE95E00E94DD2A2AE030E040EC51EDDD
:102DE00068E97BE186EE95E00E946B2B6CE286EE53
:102DF00095E00E941D2BADCF0F5F043009F0A9CFE5
:102E000029813A814B815C81A8EEB3E00E94402E7B
:102E1000698B7A8B8B8B9C8B2D813E814F81588562
:102E20000E94402E698F7A8F8B8F9C8F29853A85DF
:102E30004B855C852D8F3E8F4F8F58A32D853E850A
:102E40004F8558890E94402E6B017C0160323EE420
:102E500073078105910530F462E38CE10E94E20979
:102E600000E077CF603345E774078105910510F4E2
:102E700062E2F3CF60345CE975078105910510F4D7
:102E800066E2EBCF80E5C81683ECD806E104F104D6
:102E900010F462E1E2CF90E6C9169AEED906E10499
:102EA000F10410F465E1D9CFA0E7CA16A1E1DA0672
:102EB000A1E0EA06F10410F461E0CFCFB0EACB164E
:102EC000B6E8DB06B1E0EB06F10410F463E0C5CF31
:102ED00065E0C3CF10ED180F1A3008F03ACFE1E0EB
:102EE000F0E0EC0FFD1F24E0029FE00DF11D112426
:102EF0002081318142815381AAE0B0E00E94402EBE
:102F0000610F711D811D911D608371838283938385
:102F100020CF49885A886B887C88812C912C540159
:102F200018CF81149104A104B10489F4C301B20142
:102F30000E94510A61E070E080E090E00E94422926
:102F40001D8A1E8A1F8A188E312C22242A948D8D68
:102F50009E8DAF8DB8A188169906AA06BB06D0F43F
:102F60000E940B0A2D893E894F89588D280F311DEB
:102F7000411D511D2D8B3E8B4F8B588F381608F4F9
:102F8000382E821508F4282E3FEF831A930AA30ADD
:102F9000B30A56C0C301B20128EE33E040E050E06E
:102FA0000E94772EBA01A9012AE030E086EE95E072
:102FB0000E94C22B6CE286EE95E00E94DD2A4AE078
:102FC00050E0632D86EE95E00E94D12B6CE286EEF8
:102FD00095E00E94DD2A6D897E898F89988DA501F3
:102FE00094010E94772EBA01A9012AE030E086EE12
:102FF00095E00E94C22B6CE286EE95E00E94DD2AED
:103000004AE050E0622D86EE95E00E94D12B6CE202
:1030100086EE95E00E941D2B4C0C5D1C6E1C7F1CE7
:10302000898D9A8DAB8DBC8D84159505A605B70548
:1030300020F449885A886B887C88812C912C540113
:1030400029893A894B895C89283E334041055105DD
:1030500009F07FCEA296E2E10C94D42EACE1B0E070
:10306000E4E3F8E10C94C22E0E941F296B017C015D
:1030700081E00E94C10A14E703E0198361E0CE01F8
:1030800001960E941E0C009377050E949C0B6AEF2C
:1030900070E080E090E00E944229809177058330C3
:1030A00089F486EE95E00E941F2C892B59F40E942A
:1030B0001F296C197D098E099F096038734C894C52
:1030C0009140D8F280917705833009F44FC08FE7A3
:1030D0000E94BA090E94CD098983843511F083E0EA
:1030E0005CC00E94CD0910924A0580934B050E9456
:1030F000CD0920914A0530914B05280F311D3093A1
:103100004B0520934A050E94CD0980934C050E94EF
:10311000CD0980934D05813110F7F12C0F2D10E072
:1031200080914D0590E0880F991F0817190740F40A
:103130000E94CD09F801E25BFA4F8083F394EECF51
:1031400080E7898361E0CE0101960E941E0C83E036
:10315000809377050E949C0B62E370E080E090E032
:103160000E94422980917705833011F482E015C0D6
:103170008FE70E94BA090E94CD098983803509F042
:10318000AECF03EA15E00E94CD09F80181938F01CB
:10319000F5E00E3B1F07B9F781E06C96E8E00C9470
:1031A000DE2E80914905992787FD9095A92FB92F8B
:1031B000FC013196EB30F10508F066C0EC5CFF4F86
:1031C0000C94EF2E62E778E086EE95E00E94F92AF3
:1031D00088E893E00E94730C6AE578E086EE95E05B
:1031E0000E94F92A65E378E086EE95E00E94F92ACC
:1031F0006BE078E086EE95E00E94F92A6AEE77E0CF
:1032000086EE95E00E94F92A6DEB77E086EE95E078
:103210000E94F92A67E977E086EE95E00E94F92A94
:1032200063E777E086EE95E00E94F92A6CE477E0A8
:1032300086EE95E00E94F92A86EE95E00E94E52A46
:103240000E94B30D21C06FE277E01AC06AE077E018
:1032500017C065EF76E014C066ED76E011C062E954
:1032600076E00EC06DE776E00BC068E676E086EEAD
:1032700095E00E94F92A62E276E002C06CE076E016
:1032800086EE95E00E94F92A6AE070E080E090E026
:103290000E94422986EE95E00E941F2C892B29F07E
:1032A00086EE95E00E944C2CF5CF0895ACE1B0E09D
:1032B000ECE5F9E10C94C22E909149059F3F09F08D
:1032C00023C1482F50E0FA013A97EF36F10508F094
:1032D0000FC1E15CFF4F0C94EF2E61E172E0A0C0E2
:1032E0006DE172E086EE95E00E940B2B85E7898305
:1032F0008BE1E3EAF5E0DE01129601900D928A95EA
:10330000E1F76CE1CE0101960E941E0C0E949C0B1D
:1033100083E08093770568EC70E080E090E00E94A5
:10332000422980917705843009F0E2C08FE70E943E
:10333000BA090E94CD098983853509F0D9C06DEE9F
:1033400074E086EE95E00E94F92A6FEC74E086EE58
:1033500095E00E94F92A61EB74E096C065E372E0A3
:1033600086EE95E00E940B2B89E6898361E0CE0111
:1033700001960E941E0C0E949C0B83E080937705AF
:1033800068EC70E080E090E00E944229809177052F
:10339000843009F0ADC08FE70E94BA090E94CD09C0
:1033A00089838E010E5F1F4F7E014DE1E40EF11CFB
:1033B0000E94CD09F80181938F01EE15FF05C1F739
:1033C0008BE1FE013296A3EAB5E001900D928A9559
:1033D000E1F78981893409F08BC063E974E086EEF6
:1033E00095E00E94F92A65E774E086EE95E00E9478
:1033F000F92A67E574E048C06FE472E086EE95E074
:103400000E940B2B8EEF8093490572C0805287502B
:10341000805390914C05981708F066C06EE572E0F5
:1034200086EE95E00E940B2B63C084E180934905F2
:1034300060E274E029C085E18093490569EE73E09C
:1034400023C086E18093490562EB73E01DC087E1EC
:103450008093490568E673E017C088E180934905C9
:1034600067E573E011C089E18093490563E473E087
:103470000BC08AE1809349056EE273E005C08BE1E1
:103480008093490566E073E086EE95E00E94F92A94
:103490002FC06CEE72E086EE95E00E94F92A8091D2
:1034A000B10591E01DC066ED72E086EE95E00E94E8
:1034B000F92A8091B10592E013C061EC72E086EECA
:1034C00095E00E94F92A8091B10594E009C066EA6E
:1034D00072E086EE95E00E94F92A8091B10598E0AD
:1034E00089278093B1058FEF809349050E9454107E
:1034F00086EE95E00E941F2C892B09F45BC186EEB5
:1035000095E00E944C2CF4CF0E945311882309F4BB
:1035100051C18091E304811104C08FEF809349056C
:1035200041C140E050E060E070E084EE94E00E9431
:10353000662F40914905042F112707FD1095212F73
:10354000312FF8013197EB31F10508F01BC1E2553D
:10355000FF4F0C94EF2E552747FD509520914C05B9
:1035600030E0241735070CF40DC18B019C0101508C
:10357000110921093109003211052105310558F0E1
:10358000C0904D05EFE4F5E0F12CD12CA8E2EA2E35
:10359000415051090FC0FA01ED55FA4F6150608357
:1035A000D9C0DF0111972C9130E02417350729F09D
:1035B000F3943296FC10F5CFCBC00E2D10E020E036
:1035C00030E0061717072807390741F42081DA0190
:1035D000AD55BA4F11962C93DD24D394E394E8CFE4
:1035E0006F3F71058105910511F008F0CBC0609324
:1035F000BB05B0C06F3F71058105910511F008F062
:10360000C1C06093BC05A6C06F3F710581059105DF
:1036100011F008F0B7C06093BD059CC02091E40490
:1036200020622037E9F440E050E060E070E085EE91
:1036300094E00E94662F9B01AC01DC01CB01019755
:10364000A109B1090897A105B10508F0AEC0A4ED24
:10365000B0E30E94402E6A5E7C4A8A46954E24C0A2
:103660002636E9F440E050E060E070E085EE94E05A
:103670000E94662F9B01AC01DC01CB010197A109DF
:10368000B1090797A105B10508F08FC0A8EAB1E616
:103690000E94402E645E7C438E46944E05C06115A8
:1036A00071058105910579F08B019C010054114E43
:1036B0002D4938410138F0EF1F07FAEF2F07F2E0EC
:1036C0003F0708F05FC06093B3057093B405809323
:1036D000B5059093B6053EC06F3F71058105910514
:1036E00011F008F04FC06093B70534C08B019C0106
:1036F00001501109210931090F3F1105210531053B
:1037000008F040C06093B80525C08B019C01045CA3
:103710001940210931090D344DE114072105310506
:1037200028F47093BA056093B90514C0611571054A
:103730008105910521F48FEF8093B2050BC06134B0
:10374000710581059105F0F461506093B20502C0E6
:10375000DD20C1F08091E20481111AC080918305BF
:1037600090918405A0918505B09186050196A11DD3
:10377000B11D8093830590938405A0938505B09334
:10378000860506C060E772E086EE95E00E940B2B8E
:103790000E9449118FEF809349056AE086EE95E01B
:1037A0000E941D2B0E94541005C061E070E080E073
:1037B00090E07ACF6C96E8E00C94DE2E6AE572E039
:1037C00086EE95E00E94F92A62E472E086EE95E0CA
:1037D0000E94F92A86EE95E00E941F2C892B31F079
:1037E00086EE95E00E944C2C0E9456190E942E18DD
:1037F000823029F0833051F46DE072E002C064E25F
:1038000072E086EE95E00E94F92A08958FEF80938A
:1038100049051092E2040E945410809149058E3FA0
:1038200069F086EE95E00E941F2C892BB1F386EE9D
:1038300095E00E944C2C0E945619EFCF08950F93EB
:103840001F93109149051F3F09F0D2C0893409F434
:1038500057C000F5883309F469C058F4803309F47F
:1038600077C008F061C08B3109F440C08132B1F1FA
:10387000B9C0813409F487C030F4893309F466C0D3
:10388000803461F1AFC0823409F48EC0863409F40B
:1038900048C0A8C0823609F487C078F4883531F171
:1038A00028F48235C1F18335E1F09CC08A3509F4F2
:1038B00094C0813609F467C095C0823761F128F45D
:1038C000863679F18936E1F08DC0883779F08A370C
:1038D00009F483C0833709F085C003C061E172E059
:1038E00015C00E94840D6EE872E004C00E948D0D28
:1038F00068EA72E086EE95E00E940B2B8EEF70C0B6
:103900000E947A060E94BF0667EC72E086EE95E0A0
:103910000E940B2B67C081E00E94DF0660EE72E020
:10392000F5CF0E94FE105EC080535AC06AEF71E06E
:1039300086EE95E00E94F92A9091A20588E0890F11
:103940008871977E892B8093A2051AC089E048C0B0
:1039500067EE71E086EE95E00E94F92A8091C3053A
:103960009091C405A091C505B091C60520E18227BC
:103970008093C3059093C405A093C505B093C60575
:10398000109349052FC061ED71E086EE95E00E942D
:10399000F92A8091C3059091C405A091C505B09105
:1039A000C60540E4842710C060EC71E086EE95E027
:1039B0000E94F92A8091C3059091C405A091C50584
:1039C000B091C60520E282278093C3059093C40579
:1039D000A093C505B093C60502C00E94DE1B8FEF01
:1039E00080934905809149058E3F09F0D4C0DDC020
:1039F0000E945311882309F4D8C08091E3048111F7
:103A000004C08FEF80934905C6C040E050E060E0FD
:103A100070E084EE94E00E94662F00914905112722
:103A200007FD1095212F312FF8013197E930F1056D
:103A300008F0B4C0E753FF4F0C94EF2E8B019C01AC
:103A40000154114E2D4938410F37104F2A4F324043
:103A500008F0A4C060937F05709380058093810572
:103A60009093820577C0609383057093840580935B
:103A700085059093860581E08093E2046BC06830F1
:103A800071058105910508F089C06093870562C0C2
:103A90008B019C0101501109210931090A301105DE
:103AA0002105310508F07AC06093880553C061EBA9
:103AB00071E084EE94E00E94A03010E0009799F04D
:103AC0000E947A30009779F0183130F4E12FF0E05D
:103AD000E658FA4F87871F5F61EB71E080E090E066
:103AE0000E94A030EBCF1831A8F5E12FF0E0E658A6
:103AF000FA4F17861F5FF7CF653071058105910575
:103B000008F04CC06093A10525C08B019C010150B9
:103B10001109210931090630110521053105F0F59A
:103B20002091A205287F262B2093A20513C08B018C
:103B30009C0101501109210931090115124C214044
:103B4000310560F560937B0570937C0580937D055E
:103B500090937E058091E204811113C080918305CA
:103B600090918405A0918505B09186050196A11DCF
:103B7000B11D8093830590938405A0938505B09330
:103B800086050E9449118FEF809349056AE086EE11
:103B900095E00E941D2B0E94D11807C060E772E0DB
:103BA00086EE95E00E940B2BECCF1F910F910895AC
:103BB0008FEF809349051092E2040E94D118809102
:103BC00049058E3F69F086EE95E00E941F2C892BF7
:103BD000B1F386EE95E00E944C2C0E941F1CEFCFA3
:103BE0006AE070E080E090E00E94422986EE95E075
:103BF0000E941F2C892B29F086EE95E00E944C2C08
:103C0000F5CF0895CF93C82F682F86EE95E00E94D8
:103C1000792C90916E059C2790936E05CF91089515
:103C2000A1E0B0E0E6E1FEE10C94C82E99830E9489
:103C3000021E9981892F0E94021E2196E2E00C94B7
:103C4000E42E1F93CF93DF93182FEB0110926E0594
:103C500065EB70E086EE95E00E94590662E670E042
:103C600086EE95E00E945906812F0E94021ECE0129
:103C70000E94101EDF91CF911F91089560916E05F3
:103C800086EE95E00E94792C0895A1E2B0E0EBE485
:103C9000FEE10C94C42E7B018A018C3009F452C1E0
:103CA00008F040C0863009F4BCC018F5833009F430
:103CB00091C070F4813009F472C0823009F049C2B9
:103CC0006BE170E082E00E94211E03EA15E078C0FB
:103CD000843009F487C0853009F03BC260914D05FE
:103CE00070E0660F771F85E00E94211E0EE415E04C
:103CF00086C0893009F4A7C070F4873009F49BC0EE
:103D0000883009F026C261E070E088E00E94211E40
:103D10008091D80524C28A3009F4CAC08B3009F4D6
:103D2000F1C017C28A3609F474C1D8F4873609F491
:103D300039C138F4853609F40DC1863609F41EC13F
:103D400008C2883609F436C1893609F002C261E03A
:103D500070E089E60E94211E0E947A060E94BF063A
:103D6000F6C18D3609F4D3C138F48B3609F490C10D
:103D70008C3609F499C1EDC18E3609F4DDC1873C5A
:103D800009F0E7C161E070E087EC0E94211E81E04C
:103D90000E94021E0E943E1E10926F05E4C169E25D
:103DA00070E081E00E94211E0AE715E0F801819190
:103DB0008F010E94021EF5E0033A1F07B9F7D1C137
:103DC000F80181918F010E94021EF5E00E3B1F0752
:103DD000B9F7C7C161E070E083E00E94211E0E9434
:103DE0002E18BDC161E070E084E00E94211E81E0D8
:103DF0000E94021E0E943E1E0E946116B4C1809164
:103E00004D0590E0880F991F98012E5435402817D2
:103E1000390708F0A6C1F80181918F010E94021EA6
:103E2000EECF62E070E086E00E94211E88E893E019
:103E30000E94101E96C161E070E087E00E94211E82
:103E400080914C058CC186E6898361E0CE010196A4
:103E50000E941E0C0E949C0B83E08093770568EC07
:103E600070E080E090E00E944229809177058430E4
:103E7000D9F48FE70E94BA090E94CD09898386345C
:103E800069F460E270E089E00E94211E10E20E9465
:103E9000CD090E94021E1150D1F763C161E070E0AC
:103EA00089E00E94211E53C161E070E089E054C1A5
:103EB00069E170E08AE00E94211E1092BE05209107
:103EC00076058091C3059091C405A091C505B09178
:103ED000C605222311F0806801C08F778093C30547
:103EE0009093C405A093C505B093C6050EEB15E0ED
:103EF000F80181918F010E94021EF5E0073D1F0726
:103F0000B9F72FC161E270E08BE00E94211E809121
:103F1000AA048F3F39F08091AA0491E0980F909302
:103F2000AA0402C08091AA040E94021E10E0812F00
:103F30000E941E160E944C090E94101E1F5F103125
:103F4000B1F70FC161E070E08CE00E94211E80910A
:103F5000D70505C161E070E085E60E94211E89E277
:103F6000E816F10409F0FAC0D801EAE7F5E08D910E
:103F7000819385E0E33AF807D1F7E9C061E070E0AA
:103F800086E60E94211EEBE1EE16F10409F0E6C080
:103F9000D801E3EAF5E08D91819385E0EE3BF807E7
:103FA000D1F7D5C061E070E087E60E94211E0E9433
:103FB000840DCDC061E070E088E60E94211E85E797
:103FC00089838BE1E3EAF5E0DE01129601900D9220
:103FD0008A95E1F76CE1CE0101960E941E0C0E94C9
:103FE0009C0B83E08093770560E273E080E090E0D3
:103FF0000E94422980917705843009F0AFC08FE795
:104000000E94BA090E94CD098983853509F0A6C0AE
:104010009EC061E070E08AE60E94211E89E68983E5
:1040200061E0CE0101960E941E0C0E949C0B83E071
:104030008093770560E273E080E090E00E9442297F
:1040400080917705843009F089C08FE70E94BA0912
:104050000E94CD0989838E010E5F1F4F7E01EDE125
:10406000EE0EF11C0E94CD09F80181938F01EE152F
:10407000FF05C1F78BE1FE013296A3EAB5E001909E
:104080000D928A95E1F78981893409F067C05FC094
:1040900061E070E08BE60E94211EF8018081809330
:1040A000D8050E948D0D53C061E070E08CE60E943F
:1040B000211EF0E2EF16F10461F487E6898380E2C5
:1040C000F801DE01129601900D928A95E1F761E206
:1040D00003C087E4898361E0CE0101960E941E0C33
:1040E0000E949C0B83E0809377056CE474E080E091
:1040F00090E00E94422980917705843079F58FE71E
:104100000E94BA090E94CD09873441F520C061E0C0
:1041100070E08DE60E94211E89E1E816F104F1F4B9
:10412000D801EEEBF5E08D91819385E0E73DF8074E
:10413000D1F70E94D1130BC061E070E08EE60E94BF
:10414000211EF80180818093D7050E946E0D81E0C9
:1041500006C061E070E08AEC0E94211E80E00E94AF
:10416000021E0E943E1EA196E6E00C94E02EA0E006
:10417000B0E0EDEBF0E20C94C22ECAECD3E014E612
:1041800006E035E0F32E44E0E42E53E0D52E62E065
:10419000C62E86EE95E00E941F2C892B09F49BC049
:1041A00086EE95E00E944C2C282F80933504409198
:1041B000340450E04730510560F7FA01EE52FF4FEA
:1041C0000C94EF2E853B29F781E080933404E1CFF6
:1041D000823609F07DC0C0923404DBCF8093330473
:1041E00080933204D0923404D4CF9C01332730938F
:1041F0003104209330049091320498279093320434
:10420000E0923404C6CF382F2227409130045091D9
:104210003104242B352B30933104209330049091BA
:104220003204982790933204F092340425363105F5
:1042300008F4AFCF61E070E08CEC0E94211E81E0B9
:104240000E94021E0E943E1E43C020912E04309107
:104250002F04F901E653FC4F808390913204982794
:1042600090933204C901019690932F0480932E04F9
:1042700020913004309131048217930708F489CFDC
:104280000093340486CF8091320482130BC0609176
:104290002E0470912F044AEC53E0809133040E9465
:1042A000451E0DC062E070E08BEC0E94211E8091E3
:1042B00033040E94021E80916E050E94021EFE01C0
:1042C000812F11928A95E9F710922F0410922E04F3
:1042D000109234045ECFCDB7DEB7E8E00C94DE2E4A
:1042E00081E080936F0580916F05882349F086EE09
:1042F00095E00E941F2C892BB1F30E94B720F3CFC9
:104300000895AAE2B0E0E7E8F1E20C94C02E0E9422
:1043100013296B017C0181E00E94C10A86EE95E0C1
:104320000E941F2C892B29F086EE95E00E944C2CD0
:10433000F5CF5E98409811E072E6B72EE9E2AE2E16
:1043400003E00E9413296C197D098E099F09693CBD
:10435000710581059105E0F11123D1F10E94132926
:104360006B017C015D9A419A80ED97E00E94B6074F
:10437000B982EAE7F5E0DE0112968A2D01900D92EE
:104380008A95E1F76AE2CE0101960E941E0C5D98C3
:10439000419880E090E00E94B607009377050E9464
:1043A0009C0B62E370E080E090E00E9442298091E3
:1043B0007705843061F4009377058FE70E94BA098E
:1043C0000E94CD0911E0823419F410E001C011E01F
:1043D00082E10E94382A892BA1F411E012C05E9A72
:1043E000409A5D9A419A86EE95E00E944C2C8D3061
:1043F0009105B9F06CF40A97A1F05E9840985D9829
:10440000419886EE95E00E941F2C892B41F799CFA9
:104410008332910579F08234910579F70E947021F9
:10442000ECCF62EB71E086EE95E00E94F92A0E94E3
:10443000D81DE3CF0E946116E0CF8F929F92AF927A
:10444000BF92CF92DF92EF92FF921F93CF93DF93B1
:1044500082E10E94382A892B09F089C068EC70E05B
:1044600080E090E00E94422980E090E00E94B60740
:104470000E9413294B015C016B017C0180ECC80E8A
:1044800082E1D81EE11CF11C0E9413296C157D05E8
:104490008E059F0530F482E10E94382A892BA1F312
:1044A00064C082E10E94382A892B09F05EC080ED49
:1044B00097E00E94B6070E9413296B017C01D0E0AF
:1044C000C1E088E4880E86E2981EA11CB11C11E0B0
:1044D00082E10E94382A892B21F58C149D04AE04B8
:1044E000BF0430F480ED97E00E94B607D1E0F0CF32
:1044F0000E9413296C197D098E099F09693C710579
:104500008105910528F30E9413296B017C01C127C5
:1045100019F080ED97E002C080E090E00E94B607BD
:10452000D7CF80E090E00E94B607DD23B9F08091FC
:10453000D70590E0019665E070E00E94632E8093BD
:10454000D7050E946E0D0E94EC130E948D0D64EF42
:1045500071E080E090E00E94422909C080E00E9462
:10456000DF060E9405120E94840D0E948121DF91C6
:10457000CF911F91FF90EF90DF90CF90BF90AF90C1
:104580009F908F900895CF92DF92EF92FF9280E0FC
:104590000E941D080E94F40761E086E00E94CC2979
:1045A00061E085E00E94CC2961E08EE00E94CC2988
:1045B00061E08FE00E94CC2960E082E10E94CC297A
:1045C00060E088E00E94CC2961E088E00E94052A32
:1045D0000E949F0740E052EC61E070E086EE95E0BB
:1045E0000E94672D0E94EC130E948D0D0E94D11332
:1045F0008FEF8093AA040E94090878940E941329DF
:104600006B017C018091AA048F3F59F40E94132909
:104610006C197D098E099F09603D774081059105E0
:1046200088F380ED97E00E94B60761E082E10E9486
:10463000052A5E9A409A86EE95E00E941F2C892BEF
:1046400029F086EE95E00E944C2CF5CF6DEF72E0DC
:1046500086EE95E00E94DA2A88E893E00E94730CC7
:1046600064E173E086EE95E00E94DA2A4AE050E0C9
:1046700065E070E086EE95E00E94AA2B62E370E0B0
:1046800080E090E00E94422986EE95E00E941F2C77
:1046900004970CF186EE95E00E944C2C8234910533
:1046A000D1F486EE95E00E944C2C8E34910599F45D
:1046B00086EE95E00E944C2C8434910561F486EEE0
:1046C00095E00E944C2C819731F480E090E00E94AC
:1046D000B6070E94812140917B0550917C05609135
:1046E0007D0570917E05DB01CA010197A109B10921
:1046F0000497A105B10568F44093A904433029F457
:1047000040EA56E861E070E004C040E052EC61E04D
:1047100070E086EE95E00E94672D0E941D225E9853
:10472000409880E090E00E94B6070E94D11310925A
:10473000C9048091C30583FF11C080918F05882330
:1047400051F080919605882331F080919D05882352
:1047500011F087E001C085E08093C90480E00E94E9
:10476000C10A8091CA040E94F5090E949C0B109214
:104770003F0410923E0410923D04F12C8091D80524
:104780008F15B0F062E370E080E090E00E94422973
:1047900080ED97E00E94B60762E370E080E090E071
:1047A0000E94422980E090E00E94B607F394E6CF91
:1047B0008091A20584FF08C0982F987181E09831FC
:1047C00009F080E00E94C1118FE00E941D08FF9057
:1047D000EF90DF90CF900895EF92FF920F931F9389
:1047E000CF93DF938C016EE770E086EE95E00E9438
:1047F0005906E801F12CF0E2EF2E8E0188818D57E9
:10480000823048F46DE770E086EE95E00E9459062C
:1048100088818E2588832196F801608186EE95E057
:104820000E94792CF394F9E0FF12E7CF6EE770E075
:1048300086EE95E00E945906CDB7DEB7E6E00C940F
:10484000E02EA9E0B0E0E7E2F4E20C94C82E9091EB
:10485000CB0491110EC09EEF99838A836B8350E045
:10486000559547954C832D83198618861F821E8285
:104870002EC04091D004842F90E0B4E095958795A8
:10488000BA95E1F7242F2F7030E08217930719F1C2
:104890008DEF89831B82FE01349650E0842F90E0D7
:1048A000A4E095958795AA95E1F7242F2F7030E025
:1048B0008217930749F0DC01AF52BB4F8C91819373
:1048C000405F5F5F563051F74093D0045A83CE016A
:1048D00001960E94EC238091CB0490E0019666E063
:1048E00070E00E94632E8093CB042996E2E00C9442
:1048F000E42EA0E0B0E0EFE7F4E20C94C12E6C01EE
:104900006EE770E086EE95E00E9459068601E12C84
:10491000F12CC0E0D0E030E2B32EF801608183E8F2
:10492000860F823078F46DE770E086EE95E00E94A5
:104930005906F80160816B2570E086EE95E00E94D3
:10494000590604C086EE95E00E94792CE114F1042A
:1049500059F0F80180819E01280F311DC901C92F2E
:10496000DD27C80FD91FDD273FEFE31AF30A89E0DF
:10497000E816F10459F028E0E216F10421F48C2F36
:104980008095F60180870F5F1F4FC7CFCDB7DEB789
:10499000E9E00C94DD2EA9E0B0E0E1EDF4E20C9446
:1049A000C82EE82F362F8091CB0490E0019664E268
:1049B00070E00E94632E8093CB0458E9598350E144
:1049C0005A83813089F048F08230B9F08330D9F4CD
:1049D0008B8381EF8C833D8319C085E08B8381EFCE
:1049E0008C832F5F2D8312C08B8381EF8C8384E6B1
:1049F000489FA00111245D8309C084E08B8381EF6F
:104A00008C83ED8303C00E94FE1104C0CE01019689
:104A10000E9479242996E2E00C94E42EA2E0B0E012
:104A2000E4E1F5E20C94BD2E182F762E2A834983FB
:104A30000E941F296B017C018091E1048090CC04CD
:104A40009090CD04A090CE04B090CF042A814981EB
:104A50008823C1F0D701C60188199909AA09BB09A1
:104A60004C015D0191EE89169EE29906A104B10404
:104A700020F1241708F4422F202F672D812F0E9448
:104A8000CB2413C0D701C60188199909AA09BB090B
:104A90004C015D0191E3891695E79906A104B104E3
:104AA00060F0672D812F0E942124C092CC04D09207
:104AB000CD04E092CE04F092CF042296EDE00C9467
:104AC000D92EA2E2B0E0E7E6F5E20C94BE2E8CE02F
:104AD0000E94DC0981110FC06CE173E086EE95E065
:104AE0000E940B2B5E9A409A80E00E94C10A0E94AD
:104AF0009C0B5E98409886EE95E00E941F2C892BB7
:104B000001F186EE95E00E944C2C9091A904992326
:104B100019F00E94FF13EFCF40913E0450E09A013C
:104B20002F5F3F4F2F71332760913F0470E02617AE
:104B3000370709F3FA01E75BFB4F808320933E04BC
:104B4000DACF80917705843009F086C00E941F2952
:104B5000611571058105910549F06093BB0470935F
:104B6000BC048093BD049093BE040CC081E090E02F
:104B7000A0E0B0E08093BB049093BC04A093BD047C
:104B8000B093BE048091AD049091AE048160909387
:104B9000AE048093AD0483E0809377058FE70E9495
:104BA000BA0909E614E00E94CD09F80181938F014A
:104BB000F4E002371F07B9F720917204809169046D
:104BC000982F922796FF3BC090E49227909372040F
:104BD000982F98739833F1F410E0212F30E08091F2
:104BE0006904877090E0821793074CF11F5F209152
:104BF000A205812F90E0FC01E759FB4F24FF04C080
:104C000080810E94E011E9CF608186EE95E00E94EC
:104C1000792CE3CF8F7399F480916A048093B60462
:104C200080916B048093B40480916C048093B304EE
:104C300080916F0490E09093AC048093AB048091DA
:104C40003D04813019F482E080933D0480913D045D
:104C5000833011F410923D040E941F296B017C01E6
:104C60008091AF049091B004A091B104B091B204CE
:104C70000097A105B105C9F0A7019601281B390BC2
:104C80004A0B5B0BDA01C901883B9B40A105B105CA
:104C900060F00E940B0A8093B5041092AF0410924A
:104CA000B0041092B1041092B2048091BF049091AC
:104CB000C004A091C104B091C20446015701881AF2
:104CC000990AAA0ABB0A8AE795E00E943708861665
:104CD0009706A806B90608F4A9C0C092BF04D092EE
:104CE000C004E092C104F092C2040E945706809171
:104CF000AA048830A0F08091C3059091C405A091CA
:104D0000C505B091C6055CE1B695A79597958795C1
:104D10005A95D1F7892B8A2B8B2B09F0AEC1809144
:104D2000AA048F5F8093AA048091BB049091BC0475
:104D3000A091BD04B091BE040097A105B105F1F0AA
:104D4000C81AD90AEA0AFB0A8AE795E00E943708DE
:104D50006C157D058E059F0508F014C18091C30573
:104D600084FD04C080ED97E00E94B6071092BB045A
:104D70001092BC041092BD041092BE049091720473
:104D8000907C9093720450913E0480913F04209156
:104D90003D04581709F413C1223009F010C190588E
:104DA00090937204E091A205E770F0E0E658FC4FA2
:104DB0006081693008F0EBC0615040E04613E9C003
:104DC00080933F0487E3840F90917204892B809332
:104DD00072044093400483E080933D045D9A419ABD
:104DE000809187059091C904911138C10E94BC0A35
:104DF0008091CA040E94F509E091A205E770F0E0F5
:104E0000E658FC4F608182E794E00E94D70BE09166
:104E1000CA04EF5FE093CA04E83109F42BC1F0E063
:104E2000E658FA4F8785882309F424C10E94460C6E
:104E3000813069F58091A205887149F18091AD04B6
:104E40009091AE04880F991F9093AE048093AD04A7
:104E500083E0809377050E949C0B0E941F2960933A
:104E6000AF047093B0048093B1049093B204672BA5
:104E7000682B692B61F481E090E0A0E0B0E08093C2
:104E8000AF049093B004A093B104B093B2048091A6
:104E9000A20584FF2BC08091BB049091BC04A0911B
:104EA000BD04B091BE04892B8A2B8B2BF9F0809125
:104EB000AD049091AE048E7F0E946D09182F609111
:104EC000AB048091B6040E94F513482F612F8091A6
:104ED000B50449A30E94F5130091D805282F49A1D4
:104EE0006091B3048091B4040E940E255D984198AE
:104EF0008091C7048130C1F018F08230B1F1CBC08D
:104F000082E10E94382A892B09F0C5C081E0809394
:104F1000C7040E9413296093C3047093C404809350
:104F2000C5049093C604B7C082E10E94382A892B39
:104F300031F50E941329C090C304D090C404E090BE
:104F4000C504F090C6046C197D098E099F09693E5D
:104F500073408105910508F49EC082E08093C704E8
:104F600080ED97E00E94B60796C082E10E94382A41
:104F7000892B09F490C080E090E00E94B60710925F
:104F8000C70489C080E090E00E94B607F7CE68E0D1
:104F900014CF851709F414CF4F5F242F30E090E031
:104FA000F901EE58FB4FDC01A75BBB4F7C9170838E
:104FB000F901E05CFB4F708301968F71FFCE2430C6
:104FC000B1F42091400481E494E0A3E7B4E0FC0153
:104FD0003E2F381B321718F431913D93F9CF87E3F8
:104FE000820F90917204892B80937204F4CE809189
:104FF000C704823059F49160909372045E9A409A8B
:105000008E010F5F1F4FF12CB80111C05E984098C0
:1050100080913D04811103C081E080933D04809123
:105020003D04833069F784E080933D04E9CF8F2D00
:1050300069A37AA30E941E16F801819391938F01B0
:10504000F39469A17AA1F0E1FF12F1CF8091A2055A
:1050500043E754E087700E94BC08C0CE882309F45F
:10506000C5CE2091C80431E0320F3093C804291313
:10507000BDCE0DC01092CA04D9CE8091AA0488304A
:1050800011F45E9A409A89E08093AA04CFCE1092E0
:10509000C8048150ABCEA296ECE00C94DA2E82309C
:1050A000E8F4E82FF0E0EE0FFF1FE752FA4F7183AC
:1050B0006083813041F0809169008C7F842B8093E4
:1050C0006900E89A089580916900440F551F440FC4
:1050D000551F837F842B80936900E99A08951F925E
:1050E0000F920FB60F9211242F933F934F935F931C
:1050F0006F937F938F939F93AF93BF93EF93FF93A0
:105100008091D9059091DA05892B29F0E091D90594
:10511000F091DA050995FF91EF91BF91AF919F91C1
:105120008F917F916F915F914F913F912F910F9050
:105130000FBE0F901F9018951F920F920FB60F92EF
:1051400011242F933F934F935F936F937F938F938C
:105150009F93AF93BF93EF93FF938091DB05909163
:10516000DC05892B29F0E091DB05F091DC05099540
:10517000FF91EF91BF91AF919F918F917F916F912F
:105180005F914F913F912F910F900FBE0F901F9005
:1051900018951F920F920FB60F9211242F933F93E1
:1051A0008F939F93AF93BF938091DE059091DF051E
:1051B000A091E005B091E1053091DD0523E0230FDA
:1051C0002D3720F40196A11DB11D05C026E8230F3F
:1051D0000296A11DB11D2093DD058093DE059093FD
:1051E000DF05A093E005B093E1058091E205909181
:1051F000E305A091E405B091E5050196A11DB11D5F
:105200008093E2059093E305A093E405B093E50550
:10521000BF91AF919F918F913F912F910F900FBEB2
:105220000F901F9018952FB7F8946091DE0570913C
:10523000DF058091E0059091E1052FBF08953FB70C
:10524000F8948091E2059091E305A091E405B09176
:10525000E50526B5A89B05C02F3F19F00196A11DB5
:10526000B11D3FBF6627782F892F9A2F620F711DBE
:10527000811D911D42E0660F771F881F991F4A9577
:10528000D1F70895CF92DF92EF92FF92CF93DF9301
:105290006B017C010E941F29EB01C114D104E104C0
:1052A000F10479F00E941F296C1B7D0B683E73404E
:1052B000A0F381E0C81AD108E108F108C851DC4F19
:1052C000ECCFDF91CF91FF90EF90DF90CF900895DA
:1052D000789484B5826084BD84B5816084BD85B5D1
:1052E000826085BD85B5816085BDEEE6F0E0808198
:1052F00081608083E1E8F0E01082808182608083B9
:10530000808181608083E0E8F0E08081816080833B
:10531000E1EBF0E0808184608083E0EBF0E080816D
:1053200081608083EAE7F0E080818460808380810F
:1053300082608083808181608083808180688083B7
:105340001092C1000895833081F028F4813099F0E3
:105350008230A1F008958630A9F08730B9F084300A
:10536000D1F4809180008F7D03C0809180008F7781
:1053700080938000089584B58F7702C084B58F7DB7
:1053800084BD08958091B0008F7703C08091B000F4
:105390008F7D8093B0000895CF93DF9390E0FC0160
:1053A000ED50F44F2491FC01E95FF34F8491882381
:1053B00049F190E0880F991FFC01E15DF34FA59141
:1053C000B4918B5D934FFC01C591D4919FB761114E
:1053D00008C0F8948C91209582238C938881822335
:1053E0000AC0623051F4F8948C91322F30958323A7
:1053F0008C938881822B888304C0F8948C91822BB3
:105400008C939FBFDF91CF910895A1E0B0E0EBE0D6
:10541000FAE20C94C62E282F30E0F901E152F44F45
:105420008491F901ED50F44F1491F901E95FF34FC4
:1054300004910023C9F0882321F069830E94A329E5
:105440006981E02FF0E0EE0FFF1FEB5DF34FA591B8
:10545000B4919FB7F8948C91611103C0109581238A
:1054600001C0812B8C939FBF2196E4E00C94E22E27
:10547000CF93DF93282F30E0F901E152F44F84916C
:10548000F901ED50F44FD491F901E95FF34FC49164
:10549000CC2391F081110E94A329EC2FF0E0EE0FB4
:1054A000FF1FE55EF34FA591B4912C912D2381E070
:1054B00090E021F480E002C080E090E0DF91CF91A5
:1054C00008958E3008F08E50877020919D0190E4F1
:1054D000299F90011124822B80937C0080917A0077
:1054E000806480937A0080917A0086FDFCCF809161
:1054F00078002091790090E0922B0895A0E0B0E030
:10550000E4E8FAE20C94C22E6C017A01EB01E60E9B
:10551000F71E00E010E0CE15DF0561F06991D601BD
:10552000ED91FC910190F081E02DC6010995080FE5
:10553000191FF1CFC801CDB7DEB7E8E00C94DE2E1D
:105540006115710589F0DB010D900020E9F7AD01CF
:1055500041505109461B570BDC01ED91FC91028033
:10556000F381E02D0995089580E090E00895EF9291
:10557000FF920F931F93CF93DF938C01FB01C0E049
:10558000D0E064917F018FEFE81AF80A662361F09A
:10559000D801ED91FC910190F081E02DC8010995B1
:1055A000C80FD91FF701EDCFCE01CDB7DEB7E6E0CA
:1055B0000C94E02E0E94A02A0895DC01ED91FC914C
:1055C0000190F081E02D099508950F931F93CF93DB
:1055D000DF93EC016DE00E94DD2A8C016AE0CE01D0
:1055E0000E94DD2A800F911FDF91CF911F910F91B3
:1055F00008950F931F93CF93DF93EC010E94B72A76
:105600008C01CE010E94E52A800F911FDF91CF917E
:105610001F910F9108950F931F93CF93DF93EC0188
:105620000E94A02A8C01CE010E94E52A800F911FC2
:10563000DF91CF911F910F9108950F931F93CF93F7
:10564000DF93EC010E94DD2A8C01CE010E94E52A45
:10565000800F911FDF91CF911F910F910895A1E2CB
:10566000B0E0E5E3FBE20C94BE2E7C01C42EE52FF6
:10567000CB01D22E19A221E02D1510F02AE0D22E56
:105680008E010F5D1F4F8D2C912CA12CB12C6C2DF8
:105690007E2FA50194010E94772E8C2DD29E801919
:1056A0001124015011098A3010F4805D01C0895C19
:1056B000F8018083211531054105510521F0C22EE5
:1056C000E32FCA01E4CFB801C7010E94A02AA19626
:1056D000ECE00C94DA2EA0E0B0E0E1E7FBE20C9401
:1056E000C22EEC016A017B012115310541F4E881EC
:1056F000F9810190F081E02D642F09951DC02A30B9
:105700003105A9F477FF12C06DE20E94DD2A8C01F9
:1057100044275527BA014C195D096E097F092AE013
:10572000CE010E942F2B800F911F06C02AE0B701E7
:10573000A601CE010E942F2BCDB7DEB7E8E00C9476
:10574000DE2E9A01AB01662757FD6095762F0E94E9
:105750006B2B08950F931F93CF93DF93EC019A0166
:10576000AB01662757FD6095762F0E946B2B8C014D
:10577000CE010E94E52A800F911FDF91CF911F91EA
:105780000F9108952115310549F4DC01ED91FC914B
:105790000190F081E02D642F099508950E942F2B30
:1057A00008959A01462F50E060E070E00E94C22BFD
:1057B00008959A01AB0160E070E00E94C22B089549
:1057C0000F931F93CF93DF93EC010E94C22B8C01A8
:1057D000CE010E94E52A800F911FDF91CF911F918A
:1057E0000F9108950F931F93CF93DF93EC019A01CC
:1057F000AB0160E070E00E94C22B8C01CE010E94E0
:10580000E52A800F911FDF91CF911F910F9108958D
:105810000F931F93CF93DF93EC019A01462F50E033
:1058200060E070E00E94C22B8C01CE010E94E52A4C
:10583000800F911FDF91CF911F910F910895FC016F
:1058400024853585F901E05CFF4F80819181F90164
:10585000EE5BFF4F20813181821B930B8F73992761
:105860000895FC0184859585FC01E05CFF4F408133
:105870005181FC01EE5BFF4F2081318142175307BC
:1058800041F00190F081E02DE80FF91F808190E058
:1058900008958FEF9FEF0895FC0184859585FC01A5
:1058A000E05CFF4F40815181FC01EE5BFF4F2081A6
:1058B00031814217530779F0A081B181A80FB91F38
:1058C0008C91208131812F5F3F4F2F73332731839C
:1058D000208390E008958FEF9FEF0895FC0181A150
:1058E000882329F0A489B5898C9186FFFBCF11A26A
:1058F0000895CF93DF93FC0126853785D901A05CFD
:10590000BF4F8D919C91119701968F739927E90153
:10591000CE5BDF4F4881598184179507D9F30D90ED
:10592000BC91A02DA20FB31F6C93A685B785A05C78
:10593000BF4F11969C938E93A689B7892C9181E0D5
:1059400090E0078C02C0880F991F0A94E2F7282B79
:105950002C9381E081A30488F589E02D8081806407
:10596000808381E090E0DF91CF91089508951F92A8
:105970000F920FB60F9211242F933F934F938F9353
:105980009F93EF93FF938091C00082FD1CC04091D4
:10599000C60080918C0690918D0601968F73992791
:1059A00020918E0630918F068217930771F0E09157
:1059B0008C06F0918D06E45BF94F408390938D0641
:1059C00080938C0602C08091C600FF91EF919F9159
:1059D0008F914F913F912F910F900FBE0F901F907D
:1059E000189586EE95E00E941F2C892B11F00E94DD
:1059F000B62C08951F920F920FB60F9211242F9379
:105A00003F938F939F93EF93FF932091480630919C
:105A1000490680914A0690914B062817390731F4C0
:105A20008091C1008F7D8093C10014C0E0914A062F
:105A3000F0914B06E85FF94F208180914A069091E2
:105A40004B0601968F73992790934B0680934A06D5
:105A50002093C600FF91EF919F918F913F912F91DD
:105A60000F900FBE0F901F901895A0E0B0E0EBE3F1
:105A7000FDE20C94BE2EFC011382128288EE93E0AC
:105A8000A0E0B0E084839583A683B7838CEB93E09A
:105A9000918380837587648757874687318B208BF6
:105AA000138B028BF58AE48AD78AC68AB18EA08EC0
:105AB000938E828E8F85848F8889858F8989868F42
:105AC0008A89878F8B8980A3ECE00C94DA2ECF92A1
:105AD000DF92EF92FF92CF93DF93EC016A017B019B
:105AE000411581EE580761057105F9F0EC89FD89D2
:105AF00081E090E008A002C0880F991F0A94E2F7A5
:105B0000808360E079E08DE390E0A70196010E9438
:105B1000772E2150310941095109569547953795FE
:105B20002795211580E1380798F0EC89FD891082CE
:105B300060E874E88EE190E0A70196010E94772E5C
:105B400021503109410951095695479537952795B7
:105B5000E889F9893083EA89FB89208319A2EE89D3
:105B6000FF89408181E090E09C010C8C02C0220FF3
:105B7000331F0A94E2F7422B4083EE89FF8940816C
:105B80009C010D8C02C0220F331F0A94E2F7422BB6
:105B90004083EE89FF8940819C010E8C02C0220F58
:105BA000331F0A94E2F7422B4083EE89FF8920815C
:105BB0000F8C02C0880F991F0A94E2F78095822308
:105BC0008083DF91CF91FF90EF90DF90CF90089589
:105BD0008F929F92AF92BF92CF92DF92EF92FF92FD
:105BE0000F931F9381E08F9385E08F9387E08F93CE
:105BF00083E08F9384E08F93E6EC8E2E912CF2EC71
:105C0000AF2EB12CA1ECCA2ED12CB0ECEB2EF12C86
:105C100004EC10E025EC30E048E056E06CE476E07F
:105C200086EE95E00E94352D0F900F900F900F900B
:105C30000F901F910F91FF90EF90DF90CF90BF904A
:105C4000AF909F908F9008950E9468290E94C32270
:105C5000C1EFDCE20E9461252097E1F30E94F12C64
:105C6000F9CFA29FB001B39FC001A39F700D811D0A
:105C70001124911DB29F700D811D1124911D089555
:105C80000E94312EA59F900DB49F900DA49F800D72
:105C9000911D11240895B7FF0C94402E0E94402EB0
:105CA000821B930B0895DB018F939F930E94402EDC
:105CB000BF91AF91A29F800D911DA39F900DB29FA8
:105CC000900D1124089597FB072E16F4009407D029
:105CD00077FD09D00E94F52E07FC05D03EF4909583
:105CE00081959F4F0895709561957F4F0895A1E22A
:105CF0001A2EAA1BBB1BFD010DC0AA1FBB1FEE1F46
:105D0000FF1FA217B307E407F50720F0A21BB30B90
:105D1000E40BF50B661F771F881F991F1A9469F70C
:105D200060957095809590959B01AC01BD01CF0168
:105D30000895052E97FB1EF400940E94B02E57FD87
:105D400007D00E94772E07FC03D04EF40C94B02E9F
:105D500050954095309521953F4F4F4F5F4F089597
:105D600090958095709561957F4F8F4F9F4F0895C7
:105D70002F923F924F925F926F927F928F929F925B
:105D8000AF92BF92CF92DF92EF92FF920F931F9349
:105D9000CF93DF93CDB7DEB7CA1BDB0B0FB6F894FA
:105DA000DEBF0FBECDBF09942A88398848885F843A
:105DB0006E847D848C849B84AA84B984C884DF80AB
:105DC000EE80FD800C811B81AA81B981CE0FD11D8F
:105DD0000FB6F894DEBF0FBECDBFED010895EE0FF4
:105DE000FF1F0590F491E02D0994AA1BBB1B51E104
:105DF00007C0AA1FBB1FA617B70710F0A61BB70B3B
:105E0000881F991F5A95A9F780959095BC01CD01DF
:105E100008958F929F92AF92BF92CF92DF92EF92AE
:105E2000FF92CF93DF93EC01688179818A819B8116
:105E3000611571058105910521F464E279ED8BE529
:105E400097E02DE133EF41E050E00E94992E4901A7
:105E50005A019B01AC01A7EAB1E40E94402E6B01FC
:105E60007C01ACEEB4EFA50194010E944E2EC60E4B
:105E7000D71EE81EF91EF7FE06C081E0C81AD10839
:105E8000E10880E8F80AC882D982EA82FB82C70169
:105E9000B6019F77DF91CF91FF90EF90DF90CF9089
:105EA000BF90AF909F908F9008950E94092F089502
:105EB00086E091E00E94092F089560930601709397
:105EC0000701809308019093090108952F923F9252
:105ED0005F926F927F928F929F92AF92BF92CF927A
:105EE000DF92EF92FF920F931F93CF93DF938B017B
:105EF000EA016115710521F0DB018C9311969C93E9
:105F0000209739F09E01225031092332310508F0E3
:105F1000D8C07C016701BFEFCB1ADB0A5601F7013D
:105F20006080862D90E00E949830892B11F07601D8
:105F3000F1CFFDE26F120AC0570182E0A80EB11C3A
:105F4000D70111966C90772473940BC0BBE26B124F
:105F500007C05701E2E0AE0EB11CD70111966C905C
:105F6000712CCE018F7E892B89F4B0E36B1237C080
:105F7000F50180818F7D8835D1F46180F2E0AF0E2C
:105F8000B11C872D8260782EC0E1D0E0CA30D105E7
:105F900051F1C031D10521F0C830D10599F409C0C3
:105FA000CC24CA94DC2CEC2CAFE0FA2E22C0209733
:105FB00069F7C8E0D0E0CC24CA94DC2CEC2CFFE1DB
:105FC000FF2E17C06FEF7FEFCB019E01442737FDF7
:105FD0004095542F0E94772E69017A010AC02097BC
:105FE000A9F6CAE0D0E0E9E9CE2EDC2CEC2CE9E100
:105FF000FE2EF50160E020E030E0A9014E01AA2468
:1060000097FCA094BA2C1F0170ED572E560CA9E0F6
:10601000A51570F48FEB860D8A3118F499EC592E82
:1060200006C08FE9860D8A3148F589EA582E560C4C
:10603000852D90E08C179D070CF56F3FD9F0C216A7
:10604000D306E406F50698F0C501B4010E94532E6C
:106050009B01AC01852D90E0A0E0B0E0280F391F36
:106060004A1F5B1F281739074A075B0710F46FEFB9
:1060700001C061E03196D1016C90C5CF01151105C9
:1060800051F0662311F0319703C071FE04C03297BE
:10609000D801ED93FC9370FE07C050954095309564
:1060A00021953F4F4F4F5F4F67FF10C082E290E056
:1060B00090939106809390066FEF7FEF8FEF9FEFA5
:1060C00007C060E070E080E090E002C0B901CA0162
:1060D000DF91CF911F910F91FF90EF90DF90CF90C4
:1060E000BF90AF909F908F907F906F905F903F9008
:1060F0002F900895FC0188279927E8942191203258
:10610000E9F3293010F02E30C8F32B3241F02D3254
:1061100039F4689404C00E94CC30820F911D219103
:1061200020532A30C0F31EF4909581959F4F089517
:10613000911150C0803219F089508550D0F70895E0
:1061400048EC53E00E94A5300895FA01A191B08176
:10615000009719F41097E1F0CD01DC01CD010D900D
:10616000002011F4C00113C0FB012191222319F07A
:106170002015D9F7F3CFFB012191201519F41E92B8
:10618000119606C02223C1F70D900020A1F7D0017F
:10619000FA01A193B08308957AE0979F902D879F8D
:1061A000802D910D11240895F999FECF92BD81BDE6
:1061B000F89A992780B50895262FF999FECF1FBA2E
:1061C00092BD81BD20BD0FB6F894FA9AF99A0FBE20
:0E61D00001960895992788270895F894FFCF27
:1061DE0000009206200001000000FF0002000200F5
:1061EE000200020002000200020002000200020091
:1061FE0002000200020002000200028025000005DB
:10620E00400AA1204EA50020244EA52C2330C012FA
:10621E0000001A400AA1204EA5001B1E27522C2357
:10622E00308025000005400AA1204EA50020244EF6
:10623E00A52C2330004B000006400AD0009D4900DB
:10624E007B289D492C233000E1000005400A4501C2
:10625E00D7DC03B81E0EBF00232E48E801008A408B
:10626E000A6001555502AD1E20000023C801545886
:10627E002074696D656F75742100596573004E6FDA
:10628E00002C00386368004E2F41002C205B005D0F
:10629E002028002900486F70206368616E6E656C5F
:1062AE00200020402000456E746572696E67206183
:1062BE0064617074697665206368616E6E656C20CA
:1062CE0073656C656374696F6E2C207069636B699E
:1062DE006E673A007363616E6E6572206D6F6465F2
:1062EE00004E4F5420454E41424C45440053656E7E
:1062FE0064696E672073657474696E677320746F5A
:10630E002052580A00526573657474696E67207363
:10631E00657474696E6773206F6E2052580A00415F
:10632E00626F727465642065646974730A00696EC5
:10633E0076616C69642073656C656374696F6E0059
:10634E000D0A496E76616C696420696E70757420F1
:10635E002D2064697363617264656421070053655F
:10636E007474696E677320736176656420746F2030
:10637E00454550524F4D0A005265766572746564FC
:10638E002073657474696E67732066726F6D204535
:10639E004550524F4D0A004C6F6164656420666132
:1063AE0063746F72792064656661756C74730A002C
:1063BE004B657920616E64206368616E6E656C73E7
:1063CE002072616E646F6D697A65640A004F706544
:1063DE006E4C52536E6720545820737461727469F8
:1063EE006E672000206F6E20485720006D6F647519
:1063FE006C65206C6F636B65643F00342B34003822
:10640E0000382B340031320031322B34003136005B
:10641E0050504D0052535349005344410053434C86
:10642E0000525844005458440041494E004C4245D5
:10643E0045500053504B54524D0053425553005348
:10644E00554D44004C4C494E440000070B0C1011A6
:10645E001500B7012B032F033103350338033D031A
:10646E00B7014003440349034D0351035503590338
:10647E005D0363036A036F0374038D028D028D0245
:10648E008D02160A1322312900000000792C7E2A73
:08649E001F2C4C2C312C6E2C3C
:107E00000F92CDB7DEB7112484B714BE81FFF1D035
:107E100082E08093C00088E18093C10086E0809377
:107E2000C20080E18093C4008EE0CDD088249924E4
:107E3000CC24C394F5E0DF2EE1E1EE2E73E0F72EC3
:107E4000B6D0082F813479F4B2D08983C2D0898129
:107E5000823811F481E005C0813811F485E001C059
:107E600083E09ED09AC0823411F484E103C085344B
:107E700019F485E0B6D091C0853561F498D0082F0B
:107E800010E095D090E0982E8824802A912A880CC2
:107E9000991C82C0863521F484E0A3D080E0E1CF34
:107EA000843609F04CC083D082D0A82E80D0B82E62
:107EB00000E011E07CD0F80181938F01AE16D1F77C
:107EC00088D0FB2DF53489F4E0E0F1E00BC0F9999E
:107ED000FECF92BC81BC0894811C911C819180BD15
:107EE000FA9AF99AEA1598F358C08B2D863409F05E
:107EF00054C0F401F7BEE89507B600FCFDCFF401CD
:107F0000A0E0B1E02C9130E011968C91119790E0B7
:107F1000982F8827822B932B12960C01C7BEE895C9
:107F20001124329681E0A038B80761F7F401D7BE7A
:107F3000E89507B600FCFDCFE7BEE8952EC0843774
:107F4000F1F435D034D0182F32D0B82E42D0FB2DDA
:107F5000F63421F4F40105914F010CC0FB2DF534EA
:107F600049F4F999FECF92BC81BC0894811C911C04
:107F7000F89A00B5802F14D0115049F70EC08537FC
:107F800039F427D08EE10CD085E90AD08FE069CF93
:107F9000813511F488E017D01CD080E101D050CF9A
:107FA0009091C00095FFFCCF8093C600089580910A
:107FB000C00087FFFCCF8091C00084FD01C0A89560
:107FC0008091C6000895E0E6F0E098E19083808318
:107FD0000895EDDF803219F088E0F5DFFFCF84E10E
:107FE000DFCF1F93182FE3DF1150E9F7F2DF1F9166
:0E7FF0000895282E80E0E7DFEE27FF27099492
:027FFE0001057B
:0400000300007E007B
:00000001FF
